 KbdUs

 Timestamp is 4fb05c6c (Mon May 14 13:14:20 2012)

 Preferred load address is 10000000

 Start         Length     Name                   Class
 0001:00000000 00000004H .CRT$XCA                CODE
 0001:00000004 00000004H .CRT$XCZ                CODE
 0001:00000008 00000004H .CRT$XIA                CODE
 0001:0000000c 00000004H .CRT$XIZ                CODE
 0001:00000010 00000004H .CRT$XPA                CODE
 0001:00000014 00000004H .CRT$XPZ                CODE
 0001:00000018 00000004H .CRT$XTA                CODE
 0001:0000001c 00000004H .CRT$XTZ                CODE
 0001:00000020 000038daH .rdata                  CODE
 0001:000038fc 00000022H .rdata$debug            CODE
 0001:00003920 0000cddcH .text                   CODE
 0001:000106fc 000000dcH .xdata                  CODE
 0001:000107d8 0000003cH .idata$2                CODE
 0001:00010814 00000014H .idata$3                CODE
 0001:00010828 0000013cH .idata$4                CODE
 0001:00010964 0000007eH .idata$6                CODE
 0001:000109f0 00000232H .edata                  CODE
 0002:00000000 0000013cH .idata$5                DATA
 0002:00000140 00000880H .data                   DATA
 0002:000009c0 000004d0H .bss                    DATA
 0003:00000000 00000410H .pdata                  DATA

  Address         Publics by Value              Rva+Base       Lib:Object

 0000:00000000       ___safe_se_handler_table   00000000     <absolute>
 0000:00000000       ___safe_se_handler_count   00000000     <absolute>
 0001:00000000       __xc_a                     10001000     corelib0:crt0init.obj
 0001:00000004       __xc_z                     10001004     corelib0:crt0init.obj
 0001:00000008       __xi_a                     10001008     corelib0:crt0init.obj
 0001:0000000c       __xi_z                     1000100c     corelib0:crt0init.obj
 0001:00000010       __xp_a                     10001010     corelib0:crt0init.obj
 0001:00000014       __xp_z                     10001014     corelib0:crt0init.obj
 0001:00000018       __xt_a                     10001018     corelib0:crt0init.obj
 0001:0000001c       __xt_z                     1000101c     corelib0:crt0init.obj
 0001:00000040       ??_C@_1FE@DBIINFNI@?$AAK?$AAP?$AAP?$AAL?$AAa?$AAy?$AAo?$AAu?$AAt?$AA?3?$AA?5?$AAd?$AAa?$AAt?$AAa?$AA?5?$AAs?$AAt?$AAr?$AAu?$AAc?$AAt?$AAu?$AAr?$AAe?$AA?5?$AAs?$AAi?$AAz?$AAe?$AA?5?$AAm@ 10001040     BSPKeypad:bspkeypad.obj
 0001:00000098       ??_C@_1FK@FNONLNGN@?$AA?$CF?$AAs?$AA?3?$AA?5?$AAD?$AAE?$AAB?$AAU?$AAG?$AAC?$AAH?$AAK?$AA?5?$AAf?$AAa?$AAi?$AAl?$AAe?$AAd?$AA?5?$AAi?$AAn?$AA?5?$AAf?$AAi?$AAl?$AAe?$AA?5?$AA?$CF?$AAs?$AA?5?$AAa@ 10001098     BSPKeypad:bspkeypad.obj
 0001:000000f8       ??_C@_1KK@LGBMOGEJ@?$AAC?$AA?3?$AA?2?$AAW?$AAI?$AAN?$AAC?$AAE?$AAR?$AAO?$AAO?$AAT?$AAS?$AA?2?$AAT?$AAo?$AAp?$AAa?$AAz?$AA?2?$AAW?$AAI?$AAN?$AAC?$AAE?$AA6?$AA0?$AA0?$AA?2?$AAP?$AAL?$AAA@ 100010f8     BSPKeypad:bspkeypad.obj
 0001:000001a4       ??_C@_1O@IKMMPJPA@?$AA?9?$AA?9?$AA?$CF?$AAs?$AA?$AN?$AA?6?$AA?$AA@ 100011a4     BSPKeypad:bspkeypad.obj
 0001:000001b8       ??_C@_1II@EMPIEEJ@?$AAE?$AAn?$AAd?$AA?5?$AAo?$AAf?$AA?5?$AAI?$AAn?$AAi?$AAt?$AA?5?$AAm?$AAe?$AAt?$AAh?$AAo?$AAd?$AA?5?$AA?9?$AA?5?$AAc?$AAt?$AAr?$AAl?$AA?3?$AA?5?$AA?$CF?$AAx?$AA?5?$AA?5?$AAs@ 100011b8     BSPKeypad:bspkeypad.obj
 0001:00000240       ??_C@_1DA@LMIFJCLG@?$AA?$FL?$AAK?$AAP?$AAP?$AA?$FN?$AA?$CF?$AAs?$AA?3?$AA?5?$AA?5?$AAg?$AA_?$AAp?$AAK?$AAP?$AAP?$AA?$DN?$AA0?$AAx?$AA?$CF?$AAx?$AA?$AN?$AA?6?$AA?$AA@ 10001240     BSPKeypad:bspkeypad.obj
 0001:00000270       ??_C@_1EO@MCAICMBL@?$AA?$CF?$AAs?$AA?3?$AA?5?$AAK?$AAP?$AAP?$AA?5?$AAm?$AAe?$AAm?$AAo?$AAr?$AAy?$AA?5?$AAs?$AAp?$AAa?$AAc?$AAe?$AA?5?$AAm?$AAa?$AAp?$AAp?$AAi?$AAn?$AAg?$AA?5?$AAf?$AAa?$AAi@ 10001270     BSPKeypad:bspkeypad.obj
 0001:000002c0       ??_C@_1O@JNDDBHKG@?$AA?$CL?$AA?$CL?$AA?$CF?$AAs?$AA?$AN?$AA?6?$AA?$AA@ 100012c0     BSPKeypad:bspkeypad.obj
 0001:000002d0       ??_C@_1BM@OPAJHIMO@?$AAB?$AAS?$AAP?$AAK?$AAp?$AAp?$AAR?$AAe?$AAg?$AAI?$AAn?$AAi?$AAt?$AA?$AA@ 100012d0     BSPKeypad:bspkeypad.obj
 0001:000002ec       ??_C@_1CG@HGHEHNPB@?$AAB?$AAS?$AAP?$AAK?$AAP?$AAP?$AAG?$AAe?$AAt?$AAS?$AAc?$AAa?$AAn?$AAC?$AAo?$AAd?$AAe?$AAs?$AA?$AA@ 100012ec     BSPKeypad:bspkeypad.obj
 0001:00000314       ??_C@_1DE@KHLKCBMI@?$AAS?$AAc?$AAa?$AAn?$AA?5?$AAs?$AAe?$AAq?$AAu?$AAe?$AAn?$AAc?$AAe?$AA?5?$AAc?$AAo?$AAm?$AAp?$AAl?$AAe?$AAt?$AAe?$AAd?$AA?$AN?$AA?6?$AA?$AA@ 10001314     BSPKeypad:bspkeypad.obj
 0001:00000348       ??_C@_1DK@HBNBGJO@?$AAK?$AAe?$AAy?$AAs?$AA?5?$AAd?$AAe?$AAp?$AAr?$AAe?$AAs?$AAs?$AAe?$AAd?$AA?5?$AA?$DM?$AA?5?$AA1?$AA?5?$AAp?$AAe?$AAr?$AAi?$AAo?$AAd?$AA?4?$AA?$AN?$AA?6?$AA?$AA@ 10001348     BSPKeypad:bspkeypad.obj
 0001:00000388       ??_C@_1EG@BNNCCNDO@?$AAR?$AAe?$AAl?$AAe?$AAa?$AAs?$AAe?$AA?5?$AAi?$AAn?$AAt?$AAe?$AAr?$AAr?$AAu?$AAp?$AAt?$AA?0?$AA?5?$AAK?$AAP?$AAS?$AAR?$AA?5?$AA0?$AAx?$AA?$CF?$AA0?$AA4?$AAx?$AA?4?$AA?5@ 10001388     BSPKeypad:bspkeypad.obj
 0001:000003d0       ??_C@_1CO@CDKOJIEH@?$AAK?$AAe?$AAy?$AAp?$AAr?$AAe?$AAs?$AAs?$AA?5?$AAd?$AAe?$AAb?$AAo?$AAu?$AAn?$AAc?$AAe?$AAd?$AA?4?$AA?5?$AA?$AN?$AA?6?$AA?$AA@ 100013d0     BSPKeypad:bspkeypad.obj
 0001:00000400       ??_C@_1FM@GDGFDNMF@?$AAK?$AAe?$AAy?$AA?5?$AAp?$AAr?$AAe?$AAs?$AAs?$AAe?$AAd?$AA?0?$AA?5?$AAt?$AAe?$AAm?$AAp?$AAK?$AAP?$AAS?$AAR?$AA?5?$AA0?$AAx?$AA?$CF?$AA0?$AA4?$AAx?$AA?0?$AA?5?$AAK?$AAP@ 10001400     BSPKeypad:bspkeypad.obj
 0001:00000460       ??_C@_1FO@LAOFEAMO@?$AAK?$AAe?$AAy?$AA?5?$AAr?$AAe?$AAl?$AAe?$AAa?$AAs?$AAe?$AAd?$AA?0?$AA?5?$AAt?$AAe?$AAm?$AAp?$AAK?$AAP?$AAS?$AAR?$AA?5?$AA0?$AAx?$AA?$CF?$AA0?$AA4?$AAx?$AA?0?$AA?5?$AAK@ 10001460     BSPKeypad:bspkeypad.obj
 0001:000004c0       ??_C@_1EC@GCKBKDBM@?$AAC?$AAh?$AAa?$AAn?$AAg?$AAe?$AAd?$AA?3?$AA?5?$AAd?$AAe?$AAp?$AAr?$AAe?$AAs?$AAs?$AAe?$AAd?$AA?5?$AA?$DM?$AA?5?$AA1?$AA?5?$AAp?$AAe?$AAr?$AAi?$AAo?$AAd?$AA?4?$AA?$AN?$AA?6@ 100014c0     BSPKeypad:bspkeypad.obj
 0001:00000508       ??_C@_1EG@DODJEDOI@?$AAD?$AAe?$AAp?$AAr?$AAe?$AAs?$AAs?$AA?5?$AAi?$AAn?$AAt?$AAe?$AAr?$AAr?$AAu?$AAp?$AAt?$AA?0?$AA?5?$AAK?$AAP?$AAS?$AAR?$AA?5?$AA0?$AAx?$AA?$CF?$AA0?$AA4?$AAx?$AA?4?$AA?5@ 10001508     BSPKeypad:bspkeypad.obj
 0001:00000550       ??_C@_1FM@PDOELOIJ@?$AAB?$AAe?$AAf?$AAo?$AAr?$AAe?$AA?5?$AAs?$AAc?$AAa?$AAn?$AA?0?$AA?5?$AAt?$AAe?$AAm?$AAp?$AAK?$AAP?$AAS?$AAR?$AA?5?$AA0?$AAx?$AA?$CF?$AA0?$AA4?$AAx?$AA?0?$AA?5?$AAK?$AAP@ 10001550     BSPKeypad:bspkeypad.obj
 0001:000005ac       ??_C@_1CA@IJDBLKLM@?$AAK?$AAp?$AAp?$AAS?$AAc?$AAa?$AAn?$AAS?$AAe?$AAq?$AAu?$AAe?$AAn?$AAc?$AAe?$AA?$AA@ 100015ac     BSPKeypad:bspkeypad.obj
 0001:000005cc       ??_C@_1BM@CGKCPMCA@?$AAB?$AAS?$AAP?$AAK?$AAp?$AAp?$AAP?$AAo?$AAw?$AAe?$AAr?$AAO?$AAn?$AA?$AA@ 100015cc     BSPKeypad:bspkeypad.obj
 0001:000005e8       ??_C@_1BO@NDJBJGIF@?$AAB?$AAS?$AAP?$AAK?$AAp?$AAp?$AAP?$AAo?$AAw?$AAe?$AAr?$AAO?$AAf?$AAf?$AA?$AA@ 100015e8     BSPKeypad:bspkeypad.obj
 0001:00000608       ??_C@_1FG@GMGPANNE@?$AA?$CF?$AAs?$AA?3?$AA?5?$AAF?$AAa?$AAi?$AAl?$AAe?$AAd?$AA?5?$AAt?$AAo?$AA?5?$AAs?$AAe?$AAt?$AA?5?$AAC?$AAR?$AAM?$AA?5?$AAc?$AAl?$AAo?$AAc?$AAk?$AA?5?$AAg?$AAa?$AAt?$AAi@ 10001608     BSPKeypad:bspkeypad.obj
 0001:00000660       ??_C@_1DC@GPJMDOPB@?$AAB?$AAS?$AAP?$AAK?$AAp?$AAp?$AAS?$AAe?$AAt?$AAC?$AAl?$AAo?$AAc?$AAk?$AAG?$AAa?$AAt?$AAi?$AAn?$AAg?$AAM?$AAo?$AAd?$AAe?$AA?$AA@ 10001660     BSPKeypad:bspkeypad.obj
 0001:00000898       ??_C@_1DO@NOHFLPBO@?$AAD?$AAa?$AAt?$AAa?$AA?5?$AAs?$AAt?$AAr?$AAu?$AAc?$AAt?$AAu?$AAr?$AAe?$AA?5?$AAs?$AAi?$AAz?$AAe?$AA?5?$AAm?$AAi?$AAs?$AAm?$AAa?$AAt?$AAc?$AAh?$AA?$AN?$AA?6?$AA?$AA@ 10001898     InputLang_0409:IL_0409.obj
 0001:000008d8       ??_C@_1CI@OHCJFJPM@?$AAE?$AAR?$AAR?$AAO?$AAR?$AA?3?$AA?5?$AA?$CF?$AAs?$AA?5?$AAl?$AAi?$AAn?$AAe?$AA?5?$AA?$CF?$AAd?$AA?3?$AA?5?$AA?$AA@ 100018d8     InputLang_0409:IL_0409.obj
 0001:00000900       ??_C@_1BA@LEPJIIOK@?$AAU?$AAn?$AAk?$AAn?$AAo?$AAw?$AAn?$AA?$AA@ 10001900     InputLang_0409:IL_0409.obj
 0001:00000910       ??_C@_1IO@FLKIBFBM@?$AAC?$AA?3?$AA?2?$AAy?$AAm?$AAz?$AAk?$AAi?$AA?2?$AAp?$AAu?$AAb?$AAl?$AAi?$AAc?$AA?2?$AAC?$AAO?$AAM?$AAM?$AAO?$AAN?$AA?2?$AAo?$AAa?$AAk?$AA?2?$AAd?$AAr?$AAi?$AAv?$AAe@ 10001910     InputLang_0409:IL_0409.obj
 0001:00000ac0       ??_C@_1EO@EPMBOPPE@?$AA?$CF?$AAs?$AA?3?$AA?5?$AAM?$AAa?$AAp?$AAp?$AAe?$AAd?$AA?5?$AAv?$AAk?$AAe?$AAy?$AA?5?$AA?$CF?$AA0?$AA2?$AAx?$AA?5?$AAt?$AAo?$AA?5?$AAc?$AAh?$AAa?$AAr?$AA?5?$AA?$CF?$AA0?$AA4@ 10001ac0     LayoutManager:LayMgr.obj
 0001:00000b10       ??_C@_1FC@OFDMNFOP@?$AA?$CF?$AAs?$AA?3?$AA?5?$AAC?$AAh?$AAa?$AAn?$AAg?$AAi?$AAn?$AAg?$AA?5?$AAl?$AAi?$AAg?$AAh?$AAt?$AA?5?$AAs?$AAt?$AAa?$AAt?$AAe?$AA?5?$AAf?$AAo?$AAr?$AA?5?$AAV?$AAK?$AAe@ 10001b10     LayoutManager:LayMgr.obj
 0001:00000b68       ??_C@_1HA@EHIGJNFN@?$AAK?$AAe?$AAy?$AAb?$AAd?$AAD?$AAr?$AAi?$AAv?$AAe?$AAr?$AAV?$AAK?$AAe?$AAy?$AAT?$AAo?$AAU?$AAn?$AAi?$AAc?$AAo?$AAd?$AAe?$AA?3?$AA?5?$AAN?$AAo?$AA?5?$AAi?$AAn?$AAp@ 10001b68     LayoutManager:LayMgr.obj
 0001:00000bd8       ??_C@_1HK@JCABAAAE@?$AAC?$AA?3?$AA?2?$AAy?$AAm?$AAz?$AAk?$AAi?$AA?2?$AAp?$AAu?$AAb?$AAl?$AAi?$AAc?$AA?2?$AAC?$AAO?$AAM?$AAM?$AAO?$AAN?$AA?2?$AAo?$AAa?$AAk?$AA?2?$AAd?$AAr?$AAi?$AAv?$AAe@ 10001bd8     LayoutManager:LayMgr.obj
 0001:00000c54       ??_C@_1DC@PMCHLMJK@?$AAK?$AAe?$AAy?$AAb?$AAd?$AAD?$AAr?$AAi?$AAv?$AAe?$AAr?$AAV?$AAK?$AAe?$AAy?$AAT?$AAo?$AAU?$AAn?$AAi?$AAc?$AAo?$AAd?$AAe?$AA?$AA@ 10001c54     LayoutManager:LayMgr.obj
 0001:00000c88       ??_C@_1GA@OJOBFCAJ@?$AAV?$AAa?$AAl?$AAi?$AAd?$AAa?$AAt?$AAe?$AAI?$AAn?$AAp?$AAu?$AAt?$AAL?$AAa?$AAn?$AAg?$AAu?$AAa?$AAg?$AAe?$AA?3?$AA?5?$AAI?$AAn?$AAv?$AAa?$AAl?$AAi?$AAd?$AA?5?$AAi@ 10001c88     LayoutManager:LayMgr.obj
 0001:00000ce8       ??_C@_1BM@HMIPKDJE@?$AAV?$AAK?$AAe?$AAy?$AAT?$AAo?$AAU?$AAn?$AAi?$AAc?$AAo?$AAd?$AAe?$AA?$AA@ 10001ce8     LayoutManager:LayMgr.obj
 0001:00000d04       ??_C@_1DG@HEJMDLH@?$AA?$CF?$AAs?$AA?3?$AA?5?$AAN?$AAe?$AAw?$AA?5?$AAd?$AAe?$AAa?$AAd?$AA?5?$AAc?$AAh?$AAa?$AAr?$AA?5?$AA0?$AAx?$AA?$CF?$AA0?$AA4?$AAx?$AA?$AN?$AA?6?$AA?$AA@ 10001d04     LayoutManager:LayMgr.obj
 0001:00000d3c       ??_C@_1BM@FJHJIGLC@?$AAG?$AAe?$AAt?$AAC?$AAh?$AAa?$AAr?$AAa?$AAc?$AAt?$AAe?$AAr?$AAs?$AA?$AA@ 10001d3c     LayoutManager:LayMgr.obj
 0001:00000d58       ??_C@_1KA@IKFNAPIN@?$AAW?$AAr?$AAi?$AAt?$AAe?$AAT?$AAo?$AAC?$AAh?$AAa?$AAr?$AAB?$AAu?$AAf?$AAf?$AAe?$AAr?$AA?3?$AA?5?$AAC?$AAh?$AAa?$AAr?$AAa?$AAc?$AAt?$AAe?$AAr?$AA?5?$AAb?$AAu?$AAf@ 10001d58     LayoutManager:LayMgr.obj
 0001:00000df8       ??_C@_1EG@JFLKDNHK@?$AA?$CF?$AAs?$AA?3?$AA?5?$AAN?$AAo?$AA?5?$AAs?$AAu?$AAp?$AAp?$AAo?$AAr?$AAt?$AA?5?$AAf?$AAo?$AAr?$AA?5?$AAD?$AAK?$AAF?$AA_?$AAD?$AAE?$AAA?$AAD?$AA?5?$AAf?$AAl?$AAa?$AAg@ 10001df8     LayoutManager:LayMgr.obj
 0001:00000e40       ??_C@_1CA@HFJCLOBN@?$AAP?$AAr?$AAo?$AAc?$AAe?$AAs?$AAs?$AAD?$AAe?$AAa?$AAd?$AAK?$AAe?$AAy?$AAs?$AA?$AA@ 10001e40     LayoutManager:LayMgr.obj
 0001:00000e60       ??_C@_1HE@OBOBMNCE@?$AA?$CF?$AAs?$AA?3?$AA?5?$AAD?$AAe?$AAa?$AAd?$AA?5?$AAk?$AAe?$AAy?$AA?5?$AA?$CL?$AA?5?$AAl?$AAi?$AAg?$AAa?$AAt?$AAu?$AAr?$AAe?$AA?5?$AA0?$AAx?$AA?$CF?$AA0?$AA4?$AAx?$AA?5?$AAp@ 10001e60     LayoutManager:LayMgr.obj
 0001:00000ed8       ??_C@_1GE@GJAGNIFN@?$AAP?$AAr?$AAo?$AAc?$AAe?$AAs?$AAs?$AAL?$AAi?$AAg?$AAa?$AAt?$AAu?$AAr?$AAe?$AA?3?$AA?5?$AAT?$AAo?$AAo?$AA?5?$AAm?$AAa?$AAn?$AAy?$AA?5?$AAc?$AAh?$AAa?$AAr?$AAa?$AAc@ 10001ed8     LayoutManager:LayMgr.obj
 0001:00000f40       ??_C@_1GE@EEKLGEPK@?$AAP?$AAr?$AAo?$AAc?$AAe?$AAs?$AAs?$AAL?$AAi?$AAg?$AAa?$AAt?$AAu?$AAr?$AAe?$AA?3?$AA?5?$AAW?$AAC?$AAH?$AA_?$AAL?$AAG?$AAT?$AAR?$AA?5?$AAb?$AAu?$AAt?$AA?5?$AAn?$AAo@ 10001f40     LayoutManager:LayMgr.obj
 0001:00000fa4       ??_C@_1CA@FPHGOPGB@?$AAP?$AAr?$AAo?$AAc?$AAe?$AAs?$AAs?$AAL?$AAi?$AAg?$AAa?$AAt?$AAu?$AAr?$AAe?$AA?$AA@ 10001fa4     LayoutManager:LayMgr.obj
 0001:00000fc8       ??_C@_1FI@LMKMPEMM@?$AAM?$AAa?$AAp?$AAV?$AAi?$AAr?$AAt?$AAu?$AAa?$AAl?$AAK?$AAe?$AAy?$AA?3?$AA?5?$AAN?$AAo?$AA?5?$AAd?$AAe?$AAv?$AAi?$AAc?$AAe?$AA?5?$AAl?$AAa?$AAy?$AAo?$AAu?$AAt?$AA?5@ 10001fc8     LayoutManager:LayMgr.obj
 0001:00001020       ??_C@_1FK@KLIIDPFG@?$AAM?$AAa?$AAp?$AAV?$AAi?$AAr?$AAt?$AAu?$AAa?$AAl?$AAK?$AAe?$AAy?$AA?3?$AA?5?$AAN?$AAo?$AA?5?$AAi?$AAn?$AAp?$AAu?$AAt?$AA?5?$AAl?$AAa?$AAn?$AAg?$AAu?$AAa?$AAg?$AAe@ 10002020     LayoutManager:LayMgr.obj
 0001:0000107c       ??_C@_1BO@HJAFHJDC@?$AAS?$AAc?$AAa?$AAn?$AAC?$AAo?$AAd?$AAe?$AAT?$AAo?$AAV?$AAK?$AAe?$AAy?$AA?$AA@ 1000207c     LayoutManager:LayMgr.obj
 0001:000010a0       ??_C@_1EK@HNKEACEC@?$AAK?$AAe?$AAy?$AAb?$AAo?$AAa?$AAr?$AAd?$AA?5?$AAe?$AAv?$AAe?$AAn?$AAt?$AA?5?$AAt?$AAh?$AAr?$AAe?$AAa?$AAd?$AA?5?$AAt?$AAe?$AAr?$AAm?$AAi?$AAn?$AAa?$AAt?$AAi?$AAn@ 100020a0     LayoutManager:LayMgr.obj
 0001:000010f0       ??_C@_1IO@FAAGELJD@?$AA?$CF?$AAs?$AA?3?$AA?5?$AAP?$AAD?$AAD?$AA?5?$AA?$CF?$AAu?$AA?3?$AA?5?$AAS?$AAc?$AAa?$AAn?$AA?5?$AAc?$AAo?$AAd?$AAe?$AA?5?$AA0?$AAx?$AA?$CF?$AA0?$AA8?$AAx?$AA?5?$AA?9?$AA?$DO?$AA?5@ 100020f0     LayoutManager:LayMgr.obj
 0001:00001180       ??_C@_1HE@NMPGFJEM@?$AA?$CF?$AAs?$AA?3?$AA?5?$AAP?$AAD?$AAD?$AA?5?$AA?$CF?$AAu?$AA?3?$AA?5?$AAU?$AAs?$AAi?$AAn?$AAg?$AA?5?$AAd?$AAe?$AAv?$AAi?$AAc?$AAe?$AA?5?$AAl?$AAa?$AAy?$AAo?$AAu?$AAt?$AA?5@ 10002180     LayoutManager:LayMgr.obj
 0001:000011f8       ??_C@_1EG@GJMMGGFM@?$AA?$CF?$AAs?$AA?3?$AA?5?$AAk?$AAe?$AAy?$AAb?$AAd?$AA?5?$AA?$CF?$AAu?$AA?5?$AAs?$AAc?$AAa?$AAn?$AA?5?$AAc?$AAo?$AAd?$AAe?$AA?5?$AA0?$AAx?$AA?$CF?$AA0?$AA8?$AAx?$AA?7?$AA?$CF?$AAs@ 100021f8     LayoutManager:LayMgr.obj
 0001:00001240       ??_C@_19EPDBDPAN@?$AAD?$AAo?$AAw?$AAn?$AA?$AA@ 10002240     LayoutManager:LayMgr.obj
 0001:0000124c       ??_C@_15HJEBGHIE@?$AAU?$AAp?$AA?$AA@ 1000224c     LayoutManager:LayMgr.obj
 0001:00001258       ??_C@_1HI@HIFNONDF@?$AAK?$AAe?$AAy?$AAb?$AAo?$AAa?$AAr?$AAd?$AA?3?$AA?5?$AAK?$AAe?$AAy?$AAp?$AAr?$AAe?$AAs?$AAs?$AA?5?$AAi?$AAg?$AAn?$AAo?$AAr?$AAe?$AAd?$AA?5?$AAs?$AAi?$AAn?$AAc?$AAe@ 10002258     LayoutManager:LayMgr.obj
 0001:000012d0       ??_C@_1CK@KHMJPINM@?$AAK?$AAe?$AAy?$AAb?$AAd?$AAE?$AAv?$AAe?$AAn?$AAt?$AAT?$AAh?$AAr?$AAe?$AAa?$AAd?$AAP?$AAr?$AAo?$AAc?$AA?$AA@ 100022d0     LayoutManager:LayMgr.obj
 0001:00001300       ??_C@_1GA@ICNGPECE@?$AA?$CF?$AAs?$AA?3?$AA?5?$AAV?$AAK?$AA?3?$AA?5?$AA0?$AAx?$AA?$CF?$AA0?$AA8?$AAx?$AA?5?$AAS?$AAC?$AA?3?$AA?5?$AA0?$AAx?$AA?$CF?$AA0?$AA8?$AAx?$AA?5?$AAS?$AAh?$AAi?$AAf?$AAt?$AA?5@ 10002300     LayoutManager:LayMgr.obj
 0001:00001360       ??_C@_1HA@NLAOBOAF@?$AAK?$AAe?$AAy?$AAb?$AAo?$AAa?$AAr?$AAd?$AA?3?$AA?5?$AAR?$AAe?$AAm?$AAa?$AAp?$AAp?$AAi?$AAn?$AAg?$AA?5?$AAf?$AAu?$AAn?$AAc?$AAt?$AAi?$AAo?$AAn?$AA?5?$AAr?$AAe?$AAt@ 10002360     LayoutManager:LayMgr.obj
 0001:000013d0       ??_C@_1CE@CMMKBGEA@?$AAS?$AAe?$AAn?$AAd?$AAR?$AAe?$AAm?$AAa?$AAp?$AAp?$AAe?$AAd?$AAE?$AAv?$AAe?$AAn?$AAt?$AA?$AA@ 100023d0     LayoutManager:LayMgr.obj
 0001:000013f8       ??_C@_1HE@LCAGGIGJ@?$AAK?$AAe?$AAy?$AAb?$AAo?$AAa?$AAr?$AAd?$AA?3?$AA?5?$AAE?$AAx?$AAc?$AAe?$AAp?$AAt?$AAi?$AAo?$AAn?$AA?5?$AAi?$AAn?$AA?5?$AAd?$AAe?$AAv?$AAi?$AAc?$AAe?$AA?5?$AAl?$AAa@ 100023f8     LayoutManager:LayMgr.obj
 0001:0000146c       ??_C@_1CG@JGDFADEE@?$AAK?$AAe?$AAy?$AAb?$AAd?$AAE?$AAv?$AAe?$AAn?$AAt?$AAC?$AAa?$AAl?$AAl?$AAb?$AAa?$AAc?$AAk?$AA?$AA@ 1000246c     LayoutManager:LayMgr.obj
 0001:00001498       ??_C@_1EC@HAGJGNMN@?$AA?$CF?$AAs?$AA?3?$AA?5?$AAP?$AAr?$AAo?$AAc?$AA?5?$AAn?$AAa?$AAm?$AAe?$AA?5?$AA?$CC?$AA?$CF?$AAs?$AA?$CC?$AA?5?$AAi?$AAs?$AA?5?$AAt?$AAo?$AAo?$AA?5?$AAl?$AAo?$AAn?$AAg?$AA?$AN?$AA?6@ 10002498     LayoutManager:LayMgr.obj
 0001:000014dc       ??_C@_1CI@LMGBELGL@?$AAG?$AAe?$AAt?$AAK?$AAe?$AAy?$AAb?$AAo?$AAa?$AAr?$AAd?$AAP?$AAr?$AAo?$AAc?$AAA?$AAd?$AAd?$AAr?$AA?$AA@ 100024dc     LayoutManager:LayMgr.obj
 0001:00001508       ??_C@_1GK@PNFGDIJE@?$AA?$CF?$AAs?$AA?3?$AA?5?$AAL?$AAa?$AAy?$AAo?$AAu?$AAt?$AA?5?$AAM?$AAa?$AAn?$AAa?$AAg?$AAe?$AAr?$AA?5?$AAs?$AAu?$AAc?$AAc?$AAe?$AAs?$AAs?$AAf?$AAu?$AAl?$AAl?$AAy?$AA?5@ 10002508     LayoutManager:LayMgr.obj
 0001:00001578       ??_C@_1FM@NJGAPMGB@?$AA?$CF?$AAs?$AA?3?$AA?5?$AAL?$AAa?$AAy?$AAo?$AAu?$AAt?$AA?5?$AAM?$AAa?$AAn?$AAa?$AAg?$AAe?$AAr?$AA?5?$AAs?$AAu?$AAc?$AAc?$AAe?$AAs?$AAs?$AAf?$AAu?$AAl?$AAl?$AAy?$AA?5@ 10002578     LayoutManager:LayMgr.obj
 0001:000015d8       ??_C@_1GK@EADJFIFB@?$AAK?$AAe?$AAy?$AAb?$AAo?$AAa?$AAr?$AAd?$AA?3?$AA?5?$AAE?$AAr?$AAr?$AAo?$AAr?$AA?5?$AAs?$AAe?$AAl?$AAe?$AAc?$AAt?$AAi?$AAn?$AAg?$AA?5?$AAd?$AAe?$AAv?$AAi?$AAc?$AAe@ 100025d8     LayoutManager:LayMgr.obj
 0001:00001648       ??_C@_1ME@GIAPPCNP@?$AAK?$AAe?$AAy?$AAb?$AAo?$AAa?$AAr?$AAd?$AA?3?$AA?5?$AAC?$AAo?$AAu?$AAl?$AAd?$AA?5?$AAn?$AAo?$AAt?$AA?5?$AAa?$AAc?$AAt?$AAi?$AAv?$AAa?$AAt?$AAe?$AA?5?$AAt?$AAh?$AAe@ 10002648     LayoutManager:LayMgr.obj
 0001:00001710       ??_C@_1EI@JGJOLDCK@?$AA?$CF?$AAs?$AA?3?$AA?5?$AAF?$AAo?$AAu?$AAn?$AAd?$AA?5?$AAd?$AAe?$AAf?$AAa?$AAu?$AAl?$AAt?$AA?5?$AAi?$AAn?$AAp?$AAu?$AAt?$AA?5?$AAm?$AAe?$AAt?$AAh?$AAo?$AAd?$AA?5?$AA?$CF@ 10002710     LayoutManager:LayMgr.obj
 0001:00001758       ??_C@_1LE@PONPAOJG@?$AAK?$AAe?$AAy?$AAb?$AAo?$AAa?$AAr?$AAd?$AA?3?$AA?5?$AAD?$AAe?$AAf?$AAa?$AAu?$AAl?$AAt?$AA?5?$AAi?$AAn?$AAp?$AAu?$AAt?$AA?5?$AAm?$AAe?$AAt?$AAh?$AAo?$AAd?$AA?5?$AAs@ 10002758     LayoutManager:LayMgr.obj
 0001:00001810       ??_C@_1FA@LOAOONFK@?$AA?$CF?$AAs?$AA?3?$AA?5?$AAI?$AAn?$AAi?$AAt?$AAi?$AAa?$AAl?$AAi?$AAz?$AAe?$AAd?$AA?5?$AAP?$AAD?$AAD?$AA?5?$AA?$CF?$AAu?$AA?5?$AA?9?$AA?5?$AA?$CF?$AAs?$AA?5?$AA?$CI?$AAM?$AAa?$AAs@ 10002810     LayoutManager:LayMgr.obj
 0001:00001860       ??_C@_1GK@CFECEMAO@?$AAK?$AAe?$AAy?$AAb?$AAo?$AAa?$AAr?$AAd?$AA?3?$AA?5?$AAI?$AAn?$AAv?$AAa?$AAl?$AAi?$AAd?$AA?5?$AAk?$AAe?$AAy?$AAb?$AAd?$AA?5?$AAP?$AAD?$AAD?$AA?5?$AAi?$AAn?$AAf?$AAo@ 10002860     LayoutManager:LayMgr.obj
 0001:000018d0       ??_C@_1FC@BFKJMBD@?$AAK?$AAe?$AAy?$AAb?$AAo?$AAa?$AAr?$AAd?$AA?3?$AA?5?$AAP?$AAD?$AAD?$AA?5?$AA?$CF?$AAu?$AA?5?$AAi?$AAn?$AAi?$AAt?$AAi?$AAa?$AAl?$AAi?$AAz?$AAa?$AAt?$AAi?$AAo?$AAn?$AA?5@ 100028d0     LayoutManager:LayMgr.obj
 0001:00001924       ??_C@_1CA@PAEAFIKJ@?$AAO?$AAu?$AAt?$AA?5?$AAo?$AAf?$AA?5?$AAm?$AAe?$AAm?$AAo?$AAr?$AAy?$AA?$AN?$AA?6?$AA?$AA@ 10002924     LayoutManager:LayMgr.obj
 0001:00001948       ??_C@_1FG@KKEHCAMF@?$AAU?$AAn?$AAa?$AAb?$AAl?$AAe?$AA?5?$AAt?$AAo?$AA?5?$AAs?$AAe?$AAt?$AA?5?$AAu?$AAp?$AA?5?$AAk?$AAe?$AAy?$AAb?$AAo?$AAa?$AAr?$AAd?$AA?5?$AAl?$AAa?$AAy?$AAo?$AAu?$AAt@ 10002948     LayoutManager:LayMgr.obj
 0001:000019a0       ??_C@_11LOCGONAA@?$AA?$AA@ 100029a0     LayoutManager:LayMgr.obj
 0001:000019a4       ??_C@_1DA@ENNNKOKA@?$AAK?$AAe?$AAy?$AAb?$AAd?$AAD?$AAr?$AAi?$AAv?$AAe?$AAr?$AAI?$AAn?$AAi?$AAt?$AAi?$AAa?$AAl?$AAi?$AAz?$AAe?$AAE?$AAx?$AA?$AA@ 100029a4     LayoutManager:LayMgr.obj
 0001:000019d4       ??_C@_1CK@EJMAOEFN@?$AA?$CF?$AAs?$AA?3?$AA?5?$AAE?$AAx?$AAi?$AAt?$AAi?$AAn?$AAg?$AA?5?$AAt?$AAh?$AAr?$AAe?$AAa?$AAd?$AA?$AN?$AA?6?$AA?$AA@ 100029d4     LayoutManager:LayMgr.obj
 0001:00001a00       ??_C@_1EE@BEBODHHN@?$AA?$CF?$AAs?$AA?3?$AA?5?$AAC?$AAo?$AAu?$AAl?$AAd?$AA?5?$AAn?$AAo?$AAt?$AA?5?$AAc?$AAr?$AAe?$AAa?$AAt?$AAe?$AA?5?$AAf?$AAi?$AAl?$AAe?$AA?5?$AAo?$AAn?$AA?5?$AA?$CF?$AAs?$AA?$AN@ 10002a00     LayoutManager:LayMgr.obj
 0001:00001a48       ??_C@_1FI@JGHPMHHM@?$AA?$CF?$AAs?$AA?3?$AA?5?$AAN?$AAo?$AAt?$AAi?$AAf?$AAi?$AAc?$AAa?$AAt?$AAi?$AAo?$AAn?$AA?5?$AAf?$AAr?$AAo?$AAm?$AA?5?$AAn?$AAo?$AAn?$AA?5?$AAK?$AAB?$AAD?$AA?5?$AAd?$AAe@ 10002a48     LayoutManager:LayMgr.obj
 0001:00001aa0       ??_C@_17LIMMJKCA@?$AAK?$AAB?$AAD?$AA?$AA@ 10002aa0     LayoutManager:LayMgr.obj
 0001:00001aa8       ??_C@_1DO@KMEKPCAJ@?$AA?$CF?$AAs?$AA?3?$AA?5?$AAR?$AAe?$AAc?$AAe?$AAi?$AAv?$AAe?$AAd?$AA?5?$AA?$CF?$AAs?$AA?5?$AAn?$AAo?$AAt?$AAi?$AAf?$AAi?$AAc?$AAa?$AAt?$AAi?$AAo?$AAn?$AA?$AN?$AA?6?$AA?$AA@ 10002aa8     LayoutManager:LayMgr.obj
 0001:00001ae8       ??_C@_1GO@DOKJIHPH@?$AAK?$AAb?$AAd?$AAN?$AAo?$AAt?$AAi?$AAf?$AAi?$AAc?$AAa?$AAt?$AAi?$AAo?$AAn?$AAT?$AAh?$AAr?$AAe?$AAa?$AAd?$AA?3?$AA?5?$AAR?$AAe?$AAa?$AAd?$AAM?$AAs?$AAg?$AAQ?$AAu@ 10002ae8     LayoutManager:LayMgr.obj
 0001:00001b58       ??_C@_1IM@EMDBBKLD@?$AAK?$AAb?$AAd?$AAN?$AAo?$AAt?$AAi?$AAf?$AAi?$AAc?$AAa?$AAt?$AAi?$AAo?$AAn?$AAT?$AAh?$AAr?$AAe?$AAa?$AAd?$AA?3?$AA?5?$AAW?$AAa?$AAi?$AAt?$AAF?$AAo?$AAr?$AAM?$AAu@ 10002b58     LayoutManager:LayMgr.obj
 0001:00001be8       ??_C@_1JA@GIEDPKKC@?$AAK?$AAb?$AAd?$AAN?$AAo?$AAt?$AAi?$AAf?$AAi?$AAc?$AAa?$AAt?$AAi?$AAo?$AAn?$AAT?$AAh?$AAr?$AAe?$AAa?$AAd?$AA?3?$AA?5?$AAU?$AAn?$AAa?$AAb?$AAl?$AAe?$AA?5?$AAt?$AAo@ 10002be8     LayoutManager:LayMgr.obj
 0001:00001c78       ??_C@_1IE@GGGHHACJ@?$AAK?$AAb?$AAd?$AAN?$AAo?$AAt?$AAi?$AAf?$AAi?$AAc?$AAa?$AAt?$AAi?$AAo?$AAn?$AAT?$AAh?$AAr?$AAe?$AAa?$AAd?$AA?3?$AA?5?$AAU?$AAn?$AAa?$AAb?$AAl?$AAe?$AA?5?$AAt?$AAo@ 10002c78     LayoutManager:LayMgr.obj
 0001:00001cfc       ??_C@_1CM@HCCHLAFC@?$AAK?$AAb?$AAd?$AAN?$AAo?$AAt?$AAi?$AAf?$AAi?$AAc?$AAa?$AAt?$AAi?$AAo?$AAn?$AAT?$AAh?$AAr?$AAe?$AAa?$AAd?$AA?$AA@ 10002cfc     LayoutManager:LayMgr.obj
 0001:00001d28       ??_C@_1KG@CKCOLAOB@?$AAG?$AAe?$AAt?$AAD?$AAe?$AAf?$AAa?$AAu?$AAl?$AAt?$AAI?$AAn?$AAp?$AAu?$AAt?$AAM?$AAe?$AAt?$AAh?$AAo?$AAd?$AAN?$AAa?$AAm?$AAe?$AA?3?$AA?5?$AAN?$AAo?$AA?5?$AAv?$AAa@ 10002d28     LayoutManager:LayMgr.obj
 0001:00001dd0       ??_C@_1HE@IHAGDHOA@?$AAG?$AAe?$AAt?$AAD?$AAe?$AAf?$AAa?$AAu?$AAl?$AAt?$AAI?$AAn?$AAp?$AAu?$AAt?$AAM?$AAe?$AAt?$AAh?$AAo?$AAd?$AAN?$AAa?$AAm?$AAe?$AA?3?$AA?5?$AAN?$AAo?$AA?5?$AAv?$AAa@ 10002dd0     LayoutManager:LayMgr.obj
 0001:00001e44       ??_C@_1DE@ECMOJBFK@?$AAG?$AAe?$AAt?$AAD?$AAe?$AAf?$AAa?$AAu?$AAl?$AAt?$AAI?$AAn?$AAp?$AAu?$AAt?$AAM?$AAe?$AAt?$AAh?$AAo?$AAd?$AAN?$AAa?$AAm?$AAe?$AA?$AA@ 10002e44     LayoutManager:LayMgr.obj
 0001:00001e78       ??_C@_1EK@OEKFGJMH@?$AA?$CF?$AAs?$AA?3?$AA?5?$AAP?$AAr?$AAe?$AAl?$AAo?$AAa?$AAd?$AA?5?$AAk?$AAe?$AAy?$AA?5?$AA?$CF?$AAu?$AA?5?$AAh?$AAa?$AAs?$AA?5?$AAa?$AA?5?$AAb?$AAa?$AAd?$AA?5?$AAv?$AAa?$AAl@ 10002e78     LayoutManager:LayMgr.obj
 0001:00001ec4       ??_C@_1DE@OJAEHHEL@?$AAG?$AAe?$AAt?$AAP?$AAr?$AAe?$AAl?$AAo?$AAa?$AAd?$AAI?$AAn?$AAp?$AAu?$AAt?$AAM?$AAe?$AAt?$AAh?$AAo?$AAd?$AAN?$AAa?$AAm?$AAe?$AA?$AA@ 10002ec4     LayoutManager:LayMgr.obj
 0001:00001ef8       ??_C@_15EFLNJKHH@?$AA?$CF?$AAu?$AA?$AA@ 10002ef8     LayoutManager:LayMgr.obj
 0001:00001f00       ??_C@_1FE@FBMCGJLE@?$AA?$CF?$AAs?$AA?3?$AA?5?$AAC?$AAo?$AAu?$AAl?$AAd?$AA?5?$AAn?$AAo?$AAt?$AA?5?$AAo?$AAp?$AAe?$AAn?$AA?5?$AAP?$AAr?$AAe?$AAl?$AAo?$AAa?$AAd?$AA?5?$AAr?$AAe?$AAg?$AAi?$AAs@ 10002f00     LayoutManager:LayMgr.obj
 0001:00001f54       ??_C@_1DC@BLLENJMD@?$AAG?$AAe?$AAt?$AAP?$AAr?$AAe?$AAl?$AAo?$AAa?$AAd?$AAI?$AAn?$AAp?$AAu?$AAt?$AAM?$AAe?$AAt?$AAh?$AAo?$AAd?$AAK?$AAe?$AAy?$AA?$AA@ 10002f54     LayoutManager:LayMgr.obj
 0001:00001f8c       ??_C@_1DA@FKJDDCGN@?$AAK?$AAe?$AAy?$AAb?$AAo?$AAa?$AAr?$AAd?$AA?5?$AAL?$AAa?$AAy?$AAo?$AAu?$AAt?$AA?2?$AAP?$AAr?$AAe?$AAl?$AAo?$AAa?$AAd?$AA?$AA@ 10002f8c     LayoutManager:LayMgr.obj
 0001:00001fc0       ??_C@_1EI@KLDFCHDI@?$AA?$CF?$AAs?$AA?3?$AA?5?$AAU?$AAn?$AAn?$AAa?$AAm?$AAe?$AAd?$AA?5?$AAP?$AAr?$AAe?$AAl?$AAo?$AAa?$AAd?$AA?5?$AAv?$AAa?$AAl?$AAu?$AAe?$AA?5?$AAi?$AAs?$AA?5?$AAb?$AAa?$AAd@ 10002fc0     LayoutManager:LayMgr.obj
 0001:00002008       ??_C@_1CO@FEKOBNID@?$AAG?$AAe?$AAt?$AAP?$AAr?$AAe?$AAl?$AAo?$AAa?$AAd?$AAU?$AAn?$AAN?$AAa?$AAm?$AAe?$AAd?$AAV?$AAa?$AAl?$AAu?$AAe?$AA?$AA@ 10003008     LayoutManager:LayMgr.obj
 0001:00002038       ??_C@_1FI@IHOACNGN@?$AAI?$AAn?$AAv?$AAa?$AAl?$AAi?$AAd?$AA?5?$AAi?$AAn?$AAp?$AAu?$AAt?$AA?5?$AAl?$AAa?$AAn?$AAg?$AAu?$AAa?$AAg?$AAe?$AA?5?$AAi?$AAn?$AAf?$AAo?$AAr?$AAm?$AAa?$AAt?$AAi@ 10003038     LayoutManager:LayMgr.obj
 0001:00002090       ??_C@_1FM@PFEDIBOM@?$AA?$CF?$AAs?$AA?3?$AA?5?$AAI?$AAn?$AAp?$AAu?$AAt?$AA?5?$AAl?$AAa?$AAn?$AAg?$AAu?$AAa?$AAg?$AAe?$AA?5?$AAe?$AAn?$AAt?$AAr?$AAy?$AA?5?$AAf?$AAu?$AAn?$AAc?$AAt?$AAi?$AAo@ 10003090     LayoutManager:LayMgr.obj
 0001:000020f0       ??_C@_1EK@CFGLEGKN@?$AA?$CF?$AAs?$AA?3?$AA?5?$AAE?$AAx?$AAc?$AAe?$AAp?$AAt?$AAi?$AAo?$AAn?$AA?5?$AAi?$AAn?$AA?5?$AAe?$AAn?$AAt?$AAr?$AAy?$AA?5?$AAf?$AAu?$AAn?$AAc?$AAt?$AAi?$AAo?$AAn?$AA?5@ 100030f0     LayoutManager:LayMgr.obj
 0001:00002140       ??_C@_1FM@KEHGOGLJ@?$AA?$CF?$AAs?$AA?3?$AA?5?$AAC?$AAo?$AAu?$AAl?$AAd?$AA?5?$AAn?$AAo?$AAt?$AA?5?$AAg?$AAe?$AAt?$AA?5?$AAt?$AAh?$AAe?$AA?5?$AAa?$AAd?$AAd?$AAr?$AAe?$AAs?$AAs?$AA?5?$AAo?$AAf@ 10003140     LayoutManager:LayMgr.obj
 0001:000021a0       ??_C@_1GA@NGOLJMCD@?$AA?$CF?$AAs?$AA?3?$AA?5?$AAF?$AAa?$AAi?$AAl?$AAe?$AAd?$AA?5?$AAl?$AAo?$AAa?$AAd?$AAi?$AAn?$AAg?$AA?5?$AA?$CF?$AAs?$AA?5?$AAf?$AAo?$AAr?$AA?5?$AAi?$AAn?$AAp?$AAu?$AAt?$AA?5@ 100031a0     LayoutManager:LayMgr.obj
 0001:00002200       ??_C@_1FI@BOEFILPH@?$AA?$CF?$AAs?$AA?3?$AA?5?$AAC?$AAo?$AAu?$AAl?$AAd?$AA?5?$AAn?$AAo?$AAt?$AA?5?$AAc?$AAh?$AAa?$AAn?$AAg?$AAe?$AA?5?$AAt?$AAo?$AA?5?$AAi?$AAn?$AAp?$AAu?$AAt?$AA?5?$AAl?$AAa@ 10003200     LayoutManager:LayMgr.obj
 0001:00002258       ??_C@_1GI@LFCDMIGI@?$AA?$CF?$AAs?$AA?3?$AA?5?$AAC?$AAh?$AAa?$AAn?$AAg?$AAi?$AAn?$AAg?$AA?5?$AAf?$AAr?$AAo?$AAm?$AA?5?$AAi?$AAn?$AAp?$AAu?$AAt?$AA?5?$AAl?$AAa?$AAn?$AAg?$AAu?$AAa?$AAg?$AAe@ 10003258     LayoutManager:LayMgr.obj
 0001:000022c0       ??_C@_1CC@COBCHGHN@?$AAS?$AAe?$AAt?$AAI?$AAn?$AAp?$AAu?$AAt?$AAL?$AAa?$AAn?$AAg?$AAu?$AAa?$AAg?$AAe?$AA?$AA@ 100032c0     LayoutManager:LayMgr.obj
 0001:000022e4       ??_C@_19NGFMKOON@?$AA?$CF?$AA0?$AA8?$AAX?$AA?$AA@ 100032e4     LayoutManager:LayMgr.obj
 0001:000022f0       ??_C@_1DK@LEHEMEEF@?$AA?$CF?$AAs?$AA?3?$AA?5?$AAP?$AAr?$AAo?$AAb?$AAl?$AAe?$AAm?$AA?5?$AAr?$AAe?$AAa?$AAd?$AAi?$AAn?$AAg?$AA?5?$AAk?$AAe?$AAy?$AA?5?$AA?$CF?$AAs?$AA?$AN?$AA?6?$AA?$AA@ 100032f0     LayoutManager:LayMgr.obj
 0001:00002330       ??_C@_1EO@DNIHBIEC@?$AA?$CF?$AAs?$AA?3?$AA?5?$AAC?$AAo?$AAu?$AAl?$AAd?$AA?5?$AAn?$AAo?$AAt?$AA?5?$AAo?$AAp?$AAe?$AAn?$AA?5?$AAk?$AAe?$AAy?$AA?5?$AAf?$AAo?$AAr?$AA?5?$AAl?$AAa?$AAy?$AAo?$AAu@ 10003330     LayoutManager:LayMgr.obj
 0001:00002380       ??_C@_1DI@DHJFPFMB@?$AA?$CF?$AAs?$AA?3?$AA?5?$AAC?$AAo?$AAu?$AAl?$AAd?$AA?5?$AAn?$AAo?$AAt?$AA?5?$AAo?$AAp?$AAe?$AAn?$AA?5?$AA?$CF?$AAs?$AA?5?$AAk?$AAe?$AAy?$AA?$AN?$AA?6?$AA?$AA@ 10003380     LayoutManager:LayMgr.obj
 0001:000023b8       ??_C@_1CG@PFDANLGN@?$AAG?$AAe?$AAt?$AAI?$AAn?$AAp?$AAu?$AAt?$AAM?$AAe?$AAt?$AAh?$AAo?$AAd?$AAI?$AAn?$AAf?$AAo?$AA?$AA@ 100033b8     LayoutManager:LayMgr.obj
 0001:000023e0       ??_C@_1EI@CBNEBNIN@?$AA?$CF?$AAs?$AA?3?$AA?5?$AAN?$AAo?$AA?5?$AAm?$AAo?$AAd?$AAi?$AAf?$AAi?$AAe?$AAr?$AA?5?$AAm?$AAa?$AAt?$AAc?$AAh?$AA?5?$AAf?$AAo?$AAr?$AA?5?$AAv?$AAk?$AAe?$AAy?$AA?5?$AA?$CF@ 100033e0     LayoutManager:LayMgr.obj
 0001:00002428       ??_C@_1FA@GPKCAJJF@?$AA?$CF?$AAs?$AA?3?$AA?5?$AAE?$AAx?$AAc?$AAe?$AAe?$AAd?$AAe?$AAd?$AA?5?$AAm?$AAa?$AAx?$AA?5?$AAm?$AAo?$AAd?$AAi?$AAf?$AAi?$AAe?$AAr?$AA?5?$AAc?$AAo?$AAu?$AAn?$AAt?$AA?5@ 10003428     LayoutManager:LayMgr.obj
 0001:00002478       ??_C@_1DK@OIFLDFBG@?$AAG?$AAe?$AAn?$AAe?$AAr?$AAa?$AAt?$AAe?$AAM?$AAo?$AAd?$AAi?$AAf?$AAi?$AAe?$AAr?$AAT?$AAo?$AAS?$AAh?$AAi?$AAf?$AAt?$AAT?$AAa?$AAb?$AAl?$AAe?$AA?$AA@ 10003478     LayoutManager:LayMgr.obj
 0001:000024b8       ??_C@_1FC@JLOKMJPH@?$AA?$CF?$AAs?$AA?3?$AA?5?$AAC?$AAo?$AAu?$AAl?$AAd?$AA?5?$AAn?$AAo?$AAt?$AA?5?$AAr?$AAe?$AAa?$AAd?$AA?5?$AAv?$AAa?$AAl?$AAu?$AAe?$AA?5?$AAo?$AAf?$AA?5?$AA?$CF?$AAs?$AA?2?$AA?$CF@ 100034b8     LayoutManager:LayMgr.obj
 0001:00002510       ??_C@_1DO@PFNKHIDG@?$AA?$CF?$AAs?$AA?3?$AA?5?$AAC?$AAo?$AAu?$AAl?$AAd?$AA?5?$AAn?$AAo?$AAt?$AA?5?$AAo?$AAp?$AAe?$AAn?$AA?5?$AA?$CF?$AAs?$AA?2?$AA?$CF?$AAs?$AA?5?$AAk?$AAe?$AAy?$AA?$AN?$AA?6?$AA?$AA@ 10003510     LayoutManager:LayMgr.obj
 0001:00002550       ??_C@_1CK@DNDHAOAA@?$AAG?$AAe?$AAt?$AAI?$AAm?$AAe?$AAK?$AAe?$AAy?$AAb?$AAo?$AAa?$AAr?$AAd?$AAL?$AAa?$AAy?$AAo?$AAu?$AAt?$AA?$AA@ 10003550     LayoutManager:LayMgr.obj
 0001:0000257c       ??_C@_1CA@GLIJBCFK@?$AAK?$AAe?$AAy?$AAb?$AAo?$AAa?$AAr?$AAd?$AA?5?$AAL?$AAa?$AAy?$AAo?$AAu?$AAt?$AA?$AA@ 1000357c     LayoutManager:LayMgr.obj
 0001:000025a0       ??_C@_1FG@IKEAAOND@?$AAI?$AAn?$AAv?$AAa?$AAl?$AAi?$AAd?$AA?5?$AAd?$AAe?$AAv?$AAi?$AAc?$AAe?$AA?5?$AAl?$AAa?$AAy?$AAo?$AAu?$AAt?$AA?5?$AAi?$AAn?$AAf?$AAo?$AAr?$AAm?$AAa?$AAt?$AAi?$AAo@ 100035a0     LayoutManager:LayMgr.obj
 0001:000025f8       ??_C@_1FE@GONJHPLI@?$AA?$CF?$AAs?$AA?3?$AA?5?$AAD?$AAe?$AAv?$AAi?$AAc?$AAe?$AA?5?$AAl?$AAa?$AAy?$AAo?$AAu?$AAt?$AA?5?$AAe?$AAn?$AAt?$AAr?$AAy?$AA?5?$AAf?$AAu?$AAn?$AAc?$AAt?$AAi?$AAo?$AAn@ 100035f8     LayoutManager:LayMgr.obj
 0001:00002650       ??_C@_1FM@PGJBOEON@?$AA?$CF?$AAs?$AA?3?$AA?5?$AAU?$AAn?$AAa?$AAb?$AAl?$AAe?$AA?5?$AAt?$AAo?$AA?5?$AAl?$AAo?$AAa?$AAd?$AA?5?$AAd?$AAe?$AAv?$AAi?$AAc?$AAe?$AA?5?$AAl?$AAa?$AAy?$AAo?$AAu?$AAt@ 10003650     LayoutManager:LayMgr.obj
 0001:000026b0       ??_C@_1HO@LMMPANNC@?$AA?$CF?$AAs?$AA?3?$AA?5?$AAC?$AAo?$AAu?$AAl?$AAd?$AA?5?$AAn?$AAo?$AAt?$AA?5?$AAf?$AAi?$AAn?$AAd?$AA?5?$AAm?$AAa?$AAt?$AAc?$AAh?$AA?5?$AAP?$AAD?$AAD?$AA?5?$AA?$CF?$AAu?$AA?5@ 100036b0     LayoutManager:LayMgr.obj
 0001:00002730       ??_C@_1CA@IPKHFBAD@?$AAS?$AAe?$AAt?$AAD?$AAe?$AAv?$AAi?$AAc?$AAe?$AAL?$AAa?$AAy?$AAo?$AAu?$AAt?$AA?$AA@ 10003730     LayoutManager:LayMgr.obj
 0001:00002750       ??_C@_1FE@GAKCPDEP@?$AA?$CF?$AAs?$AA?3?$AA?5?$AAF?$AAa?$AAi?$AAl?$AAe?$AAd?$AA?5?$AAl?$AAo?$AAa?$AAd?$AAi?$AAn?$AAg?$AA?5?$AAd?$AAe?$AAv?$AAi?$AAc?$AAe?$AA?5?$AAl?$AAa?$AAy?$AAo?$AAu?$AAt@ 10003750     LayoutManager:LayMgr.obj
 0001:000027a4       ??_C@_1CK@LFKCMCDI@?$AAG?$AAe?$AAt?$AAD?$AAe?$AAv?$AAi?$AAc?$AAe?$AAL?$AAa?$AAy?$AAo?$AAu?$AAt?$AAE?$AAn?$AAt?$AAr?$AAy?$AA?$AA@ 100037a4     LayoutManager:LayMgr.obj
 0001:000027d0       ??_C@_1HC@KKNGAHGA@?$AA?$CF?$AAs?$AA?3?$AA?5?$AAF?$AAo?$AAu?$AAn?$AAd?$AA?5?$AAd?$AAe?$AAv?$AAi?$AAc?$AAe?$AA?5?$AAl?$AAa?$AAy?$AAo?$AAu?$AAt?$AA?5?$AAm?$AAa?$AAt?$AAc?$AAh?$AA?5?$AAf?$AAo@ 100037d0     LayoutManager:LayMgr.obj
 0001:00002848       ??_C@_1HG@CODMDNMO@?$AA?$CF?$AAs?$AA?3?$AA?5?$AAC?$AAo?$AAu?$AAl?$AAd?$AA?5?$AAn?$AAo?$AAt?$AA?5?$AAf?$AAi?$AAn?$AAd?$AA?5?$AAa?$AA?5?$AAd?$AAe?$AAv?$AAi?$AAc?$AAe?$AA?5?$AAl?$AAa?$AAy?$AAo@ 10003848     LayoutManager:LayMgr.obj
 0001:000028c0       ??_C@_1FG@HNPBMFMF@?$AA?$CF?$AAs?$AA?3?$AA?5?$AAN?$AAo?$AA?5?$AAd?$AAe?$AAv?$AAi?$AAc?$AAe?$AA?5?$AAl?$AAa?$AAy?$AAo?$AAu?$AAt?$AA?5?$AAs?$AAu?$AAb?$AAk?$AAe?$AAy?$AA?5?$AAf?$AAo?$AAu?$AAn@ 100038c0     LayoutManager:LayMgr.obj
 0001:00002918       ??_C@_1CG@JNFKBALO@?$AAS?$AAe?$AAl?$AAe?$AAc?$AAt?$AAD?$AAe?$AAv?$AAi?$AAc?$AAe?$AAL?$AAa?$AAy?$AAo?$AAu?$AAt?$AA?$AA@ 10003918     LayoutManager:LayMgr.obj
 0001:00002940       ??_C@_1FO@GBIOBLJG@?$AA?$CF?$AAs?$AA?3?$AA?5?$AAE?$AAr?$AAr?$AAo?$AAr?$AA?5?$AAi?$AAn?$AA?5?$AAd?$AAe?$AAv?$AAi?$AAc?$AAe?$AA?5?$AAl?$AAa?$AAy?$AAo?$AAu?$AAt?$AA?5?$AAe?$AAn?$AAt?$AAr?$AAy@ 10003940     LayoutManager:LayMgr.obj
 0001:000029a0       ??_C@_1CO@OIGNLNDP@?$AAD?$AAe?$AAv?$AAi?$AAc?$AAe?$AAL?$AAa?$AAy?$AAo?$AAu?$AAt?$AAM?$AAa?$AAt?$AAc?$AAh?$AAe?$AAs?$AAP?$AAD?$AAD?$AA?$AA@ 100039a0     LayoutManager:LayMgr.obj
 0001:000029d0       ??_C@_1M@LLCLNBHO@?$AA?$CF?$AAs?$AA_?$AA?$CF?$AAs?$AA?$AA@ 100039d0     LayoutManager:LayMgr.obj
 0001:000029dc       ??_C@_1M@FKDMEONL@?$AA?9?$AA?$CF?$AAs?$AA?$AN?$AA?6?$AA?$AA@ 100039dc     LayoutManager:LayMgr.obj
 0001:000029e8       ??_C@_1M@LFABOLDL@?$AA?$CL?$AA?$CF?$AAs?$AA?$AN?$AA?6?$AA?$AA@ 100039e8     LayoutManager:LayMgr.obj
 0001:000029f4       ??_C@_1DC@IFJFLG@?$AAL?$AAa?$AAy?$AAo?$AAu?$AAt?$AAM?$AAg?$AAr?$AAG?$AAe?$AAt?$AAK?$AAe?$AAy?$AAb?$AAo?$AAa?$AAr?$AAd?$AAT?$AAy?$AAp?$AAe?$AA?$AA@ 100039f4     LayoutManager:LayMgr.obj
 0001:00002a28       ??_C@_1FA@KNOLPHGM@?$AA?$CF?$AAs?$AA?3?$AA?5?$AAM?$AAu?$AAs?$AAt?$AA?5?$AAb?$AAe?$AA?5?$AAc?$AAa?$AAl?$AAl?$AAe?$AAd?$AA?5?$AAw?$AAi?$AAt?$AAh?$AA?5?$AAi?$AAd?$AAT?$AAh?$AAr?$AAe?$AAa?$AAd@ 10003a28     LayoutManager:LayMgr.obj
 0001:00002a78       ??_C@_1DG@IKNCCLA@?$AAL?$AAa?$AAy?$AAo?$AAu?$AAt?$AAM?$AAg?$AAr?$AAG?$AAe?$AAt?$AAK?$AAe?$AAy?$AAb?$AAo?$AAa?$AAr?$AAd?$AAL?$AAa?$AAy?$AAo?$AAu?$AAt?$AA?$AA@ 10003a78     LayoutManager:LayMgr.obj
 0001:00002ab0       ??_C@_1DO@DPIGDLGA@?$AAL?$AAa?$AAy?$AAo?$AAu?$AAt?$AAM?$AAg?$AAr?$AAG?$AAe?$AAt?$AAK?$AAe?$AAy?$AAb?$AAo?$AAa?$AAr?$AAd?$AAL?$AAa?$AAy?$AAo?$AAu?$AAt?$AAN?$AAa?$AAm?$AAe?$AA?$AA@ 10003ab0     LayoutManager:LayMgr.obj
 0001:00002af0       ??_C@_1EM@DEAGOFCP@?$AA?$CF?$AAs?$AA?3?$AA?5?$AAB?$AAu?$AAf?$AAf?$AAe?$AAr?$AA?5?$AAs?$AAi?$AAz?$AAe?$AA?5?$AAi?$AAs?$AA?5?$AAn?$AAo?$AAt?$AA?5?$AAl?$AAa?$AAr?$AAg?$AAe?$AA?5?$AAe?$AAn?$AAo@ 10003af0     LayoutManager:LayMgr.obj
 0001:00002b3c       ??_C@_1DO@DJOPKDPJ@?$AAL?$AAa?$AAy?$AAo?$AAu?$AAt?$AAM?$AAg?$AAr?$AAG?$AAe?$AAt?$AAK?$AAe?$AAy?$AAb?$AAo?$AAa?$AAr?$AAd?$AAL?$AAa?$AAy?$AAo?$AAu?$AAt?$AAL?$AAi?$AAs?$AAt?$AA?$AA@ 10003b3c     LayoutManager:LayMgr.obj
 0001:00002b80       ??_C@_1GO@LPEEAFIF@?$AA?$CF?$AAs?$AA?3?$AA?5?$AAS?$AAu?$AAc?$AAc?$AAe?$AAs?$AAs?$AAf?$AAu?$AAl?$AAl?$AAy?$AA?5?$AAl?$AAo?$AAa?$AAd?$AAe?$AAd?$AA?5?$AAl?$AAa?$AAy?$AAo?$AAu?$AAt?$AA?5?$AA?$CF@ 10003b80     LayoutManager:LayMgr.obj
 0001:00002bf0       ??_C@_1GE@FCKLEHDD@?$AA?$CF?$AAs?$AA?3?$AA?5?$AAC?$AAo?$AAu?$AAl?$AAd?$AA?5?$AAn?$AAo?$AAt?$AA?5?$AAs?$AAe?$AAt?$AA?5?$AAd?$AAe?$AAf?$AAa?$AAu?$AAl?$AAt?$AA?5?$AAv?$AAa?$AAl?$AAu?$AAe?$AA?5@ 10003bf0     LayoutManager:LayMgr.obj
 0001:00002c58       ??_C@_1EM@MEIACPAD@?$AA?$CF?$AAs?$AA?3?$AA?5?$AAC?$AAo?$AAu?$AAl?$AAd?$AA?5?$AAn?$AAo?$AAt?$AA?5?$AAc?$AAr?$AAe?$AAa?$AAt?$AAe?$AA?5?$AAp?$AAr?$AAe?$AAl?$AAo?$AAa?$AAd?$AA?5?$AAk?$AAe?$AAy@ 10003c58     LayoutManager:LayMgr.obj
 0001:00002ca8       ??_C@_1EC@OHHNMJOD@?$AA?$CF?$AAs?$AA?3?$AA?5?$AAC?$AAo?$AAu?$AAl?$AAd?$AA?5?$AAn?$AAo?$AAt?$AA?5?$AAo?$AAp?$AAe?$AAn?$AA?5?$AAp?$AAr?$AAe?$AAl?$AAo?$AAa?$AAd?$AA?5?$AAk?$AAe?$AAy?$AA?$AN?$AA?6@ 10003ca8     LayoutManager:LayMgr.obj
 0001:00002cf0       ??_C@_1GA@BALBINBG@?$AA?$CF?$AAs?$AA?3?$AA?5?$AAC?$AAo?$AAu?$AAl?$AAd?$AA?5?$AAn?$AAo?$AAt?$AA?5?$AAf?$AAi?$AAn?$AAd?$AA?5?$AAa?$AAn?$AA?5?$AAa?$AAv?$AAa?$AAi?$AAl?$AAa?$AAb?$AAl?$AAe?$AA?5@ 10003cf0     LayoutManager:LayMgr.obj
 0001:00002d50       ??_C@_1EE@JFJJNEJC@?$AA?$CF?$AAs?$AA?3?$AA?5?$AAL?$AAa?$AAy?$AAo?$AAu?$AAt?$AA?5?$AA?$CF?$AAs?$AA?5?$AAi?$AAs?$AA?5?$AAa?$AAl?$AAr?$AAe?$AAa?$AAd?$AAy?$AA?5?$AAl?$AAo?$AAa?$AAd?$AAe?$AAd?$AA?$AN@ 10003d50     LayoutManager:LayMgr.obj
 0001:00002d94       ??_C@_1CM@BKEFHEAE@?$AA?$CF?$AAs?$AA?3?$AA?5?$AAF?$AAo?$AAu?$AAn?$AAd?$AA?5?$AAl?$AAa?$AAy?$AAo?$AAu?$AAt?$AA?5?$AA?$CF?$AAs?$AA?$AN?$AA?6?$AA?$AA@ 10003d94     LayoutManager:LayMgr.obj
 0001:00002dc0       ??_C@_1FC@MCCKLOEL@?$AA?$CF?$AAs?$AA?3?$AA?5?$AAR?$AAe?$AAq?$AAu?$AAe?$AAs?$AAt?$AAe?$AAd?$AA?5?$AAl?$AAa?$AAy?$AAo?$AAu?$AAt?$AA?5?$AA?$CF?$AAs?$AA?5?$AAd?$AAo?$AAe?$AAs?$AA?5?$AAn?$AAo?$AAt@ 10003dc0     LayoutManager:LayMgr.obj
 0001:00002e18       ??_C@_1FA@KAMPNMAH@?$AA?$CF?$AAs?$AA?3?$AA?5?$AAK?$AAe?$AAy?$AAb?$AAo?$AAa?$AAr?$AAd?$AA?5?$AAl?$AAa?$AAy?$AAo?$AAu?$AAt?$AA?5?$AA?$CF?$AAs?$AA?5?$AAd?$AAo?$AAe?$AAs?$AA?5?$AAn?$AAo?$AAt?$AA?5@ 10003e18     LayoutManager:LayMgr.obj
 0001:00002e68       ??_C@_1DE@OEKJAIHK@?$AA?$CF?$AAs?$AA?3?$AA?5?$AA?$CF?$AAs?$AA?5?$AAi?$AAs?$AA?5?$AAa?$AAn?$AA?5?$AAi?$AAn?$AAv?$AAa?$AAl?$AAi?$AAd?$AA?5?$AAi?$AAd?$AA?$AN?$AA?6?$AA?$AA@ 10003e68     LayoutManager:LayMgr.obj
 0001:00002e9c       ??_C@_1DI@JHLFHMPL@?$AAL?$AAa?$AAy?$AAo?$AAu?$AAt?$AAM?$AAg?$AAr?$AAL?$AAo?$AAa?$AAd?$AAK?$AAe?$AAy?$AAb?$AAo?$AAa?$AAr?$AAd?$AAL?$AAa?$AAy?$AAo?$AAu?$AAt?$AA?$AA@ 10003e9c     LayoutManager:LayMgr.obj
 0001:00002ed8       ??_C@_1LO@CODLIIHA@?$AA?$CF?$AAs?$AA?3?$AA?5?$AAF?$AAa?$AAi?$AAl?$AAu?$AAr?$AAe?$AA?5?$AAs?$AAe?$AAt?$AAt?$AAi?$AAn?$AAg?$AA?5?$AAd?$AAe?$AAv?$AAi?$AAc?$AAe?$AA?5?$AAl?$AAa?$AAy?$AAo?$AAu@ 10003ed8     LayoutManager:LayMgr.obj
 0001:00002f98       ??_C@_1KO@BLOFMLMO@?$AA?$CF?$AAs?$AA?3?$AA?5?$AAF?$AAa?$AAi?$AAl?$AAu?$AAr?$AAe?$AA?5?$AAs?$AAe?$AAt?$AAt?$AAi?$AAn?$AAg?$AA?5?$AAi?$AAn?$AAp?$AAu?$AAt?$AA?5?$AAl?$AAa?$AAn?$AAg?$AAu?$AAa@ 10003f98     LayoutManager:LayMgr.obj
 0001:00003048       ??_C@_1DO@NIMCJCOO@?$AA?$CF?$AAs?$AA?3?$AA?5?$AAC?$AAa?$AAl?$AAl?$AAe?$AAd?$AA?5?$AAw?$AAi?$AAt?$AAh?$AA?5?$AAh?$AAk?$AAl?$AA?5?$AA?$DN?$AA?5?$AA0?$AAx?$AA?$CF?$AA0?$AA8?$AAx?$AA?$AN?$AA?6?$AA?$AA@ 10004048     LayoutManager:LayMgr.obj
 0001:00003088       ??_C@_1EA@FIGMDCGA@?$AAL?$AAa?$AAy?$AAo?$AAu?$AAt?$AAM?$AAg?$AAr?$AAA?$AAc?$AAt?$AAi?$AAv?$AAa?$AAt?$AAe?$AAK?$AAe?$AAy?$AAb?$AAo?$AAa?$AAr?$AAd?$AAL?$AAa?$AAy?$AAo?$AAu?$AAt?$AA?$AA@ 10004088     LayoutManager:LayMgr.obj
 0001:000030c8       ??_C@_1EM@JGHMPAIA@?$AAL?$AAa?$AAy?$AAo?$AAu?$AAt?$AA?5?$AAM?$AAa?$AAn?$AAa?$AAg?$AAe?$AAr?$AA?5?$AA?3?$AA?5?$AAD?$AAL?$AAL?$AA_?$AAP?$AAR?$AAO?$AAC?$AAE?$AAS?$AAS?$AA_?$AAA?$AAT?$AAT@ 100040c8     LayoutManager:LayMgr.obj
 0001:00003118       ??_C@_1EC@PDDNOLEO@?$AAK?$AAe?$AAr?$AAn?$AAe?$AAl?$AA?5?$AAP?$AAr?$AAo?$AAf?$AAi?$AAl?$AAe?$AAr?$AA?5?$AAm?$AAo?$AAd?$AAe?$AA?3?$AA?5?$AAB?$AAu?$AAf?$AAf?$AAe?$AAr?$AAe?$AAd?$AA?$AN?$AA?6@ 10004118     LayoutManager:profiler.obj
 0001:0000315c       ??_C@_1DM@LDFFLEGF@?$AAK?$AAe?$AAr?$AAn?$AAe?$AAl?$AA?5?$AAP?$AAr?$AAo?$AAf?$AAi?$AAl?$AAe?$AAr?$AA?5?$AAm?$AAo?$AAd?$AAe?$AA?3?$AA?5?$AAC?$AAe?$AAL?$AAo?$AAg?$AA?$AN?$AA?6?$AA?$AA@ 1000415c     LayoutManager:profiler.obj
 0001:00003198       ??_C@_1EG@OLMAKGJN@?$AAK?$AAe?$AAr?$AAn?$AAe?$AAl?$AA?5?$AAP?$AAr?$AAo?$AAf?$AAi?$AAl?$AAe?$AAr?$AA?5?$AAm?$AAo?$AAd?$AAe?$AA?3?$AA?5?$AAU?$AAn?$AAb?$AAu?$AAf?$AAf?$AAe?$AAr?$AAe?$AAd@ 10004198     LayoutManager:profiler.obj
 0001:000031e0       ??_C@_1BE@MPEJEKEH@?$AAK?$AAP?$AAP?$AAL?$AAa?$AAy?$AAo?$AAu?$AAt?$AA?$AA@ 100041e0     Keypad_mx25_topaz_v1:kbd.obj
 0001:000031f4       ??_C@_1DO@MEANBKIH@?$AAC?$AAo?$AAu?$AAl?$AAd?$AA?5?$AAn?$AAo?$AAt?$AA?5?$AAi?$AAn?$AAi?$AAt?$AAi?$AAa?$AAl?$AAi?$AAz?$AAe?$AA?5?$AAk?$AAe?$AAy?$AAp?$AAa?$AAd?$AA?4?$AA?$AN?$AA?6?$AA?$AA@ 100041f4     Keypad_mx25_topaz_v1:kbd.obj
 0001:00003238       ??_C@_1LO@FOHPJJDD@?$AAC?$AA?3?$AA?2?$AAW?$AAI?$AAN?$AAC?$AAE?$AAR?$AAO?$AAO?$AAT?$AAS?$AA?2?$AAT?$AAo?$AAp?$AAa?$AAz?$AA?2?$AAW?$AAI?$AAN?$AAC?$AAE?$AA6?$AA0?$AA0?$AA?2?$AAP?$AAL?$AAA@ 10004238     Keypad_mx25_topaz_v1:kbd.obj
 0001:000032f8       ??_C@_1DG@BACDDNAK@?$AA?$CF?$AAs?$AA?3?$AA?5?$AAI?$AAn?$AAi?$AAt?$AAi?$AAa?$AAl?$AAi?$AAz?$AAe?$AA?5?$AAK?$AAP?$AAP?$AA?5?$AAI?$AAD?$AA?5?$AA?$CF?$AAu?$AA?$AN?$AA?6?$AA?$AA@ 100042f8     Keypad_mx25_topaz_v1:kbd.obj
 0001:00003330       ??_C@_1BE@MFGBOMPO@?$AAK?$AAP?$AAP?$AA_?$AAE?$AAn?$AAt?$AAr?$AAy?$AA?$AA@ 10004330     Keypad_mx25_topaz_v1:kbd.obj
 0001:00003344       ??_C@_1CM@CNFNOMMH@?$AAK?$AAe?$AAy?$AAb?$AAd?$AAP?$AAd?$AAd?$AA_?$AAP?$AAo?$AAw?$AAe?$AAr?$AAH?$AAa?$AAn?$AAd?$AAl?$AAe?$AAr?$AA?$AA@ 10004344     Keypad_mx25_topaz_v1:keypad.obj
 0001:00003370       ??_C@_1CC@NCEIAIOE@?$AAK?$AAp?$AAp?$AAI?$AAs?$AAr?$AAT?$AAh?$AAr?$AAe?$AAa?$AAd?$AAP?$AAr?$AAo?$AAc?$AA?$AA@ 10004370     Keypad_mx25_topaz_v1:keypad.obj
 0001:00003394       ??_C@_1DG@MPBOBHG@?$AA?$CF?$AAs?$AA?3?$AA?5?$AAk?$AAe?$AAy?$AAp?$AAa?$AAd?$AA?5?$AAe?$AAv?$AAe?$AAn?$AAt?$AAs?$AA?5?$AA0?$AAx?$AA?$CF?$AA0?$AA8?$AAx?$AA?$AN?$AA?6?$AA?$AA@ 10004394     Keypad_mx25_topaz_v1:keypad.obj
 0001:000033d0       ??_C@_1FA@LIPICKON@?$AA?$CF?$AAs?$AA?3?$AA?5?$AAe?$AAv?$AAe?$AAn?$AAt?$AA?5?$AA0?$AAx?$AA?$CF?$AA0?$AA8?$AAx?$AA?3?$AA?5?$AAS?$AAc?$AAa?$AAn?$AAC?$AAo?$AAd?$AAe?$AA?5?$AA0?$AAx?$AA?$CF?$AA0?$AA8@ 100043d0     Keypad_mx25_topaz_v1:keypad.obj
 0001:00003420       ??_C@_1ME@KIMFCGGN@?$AAC?$AA?3?$AA?2?$AAW?$AAI?$AAN?$AAC?$AAE?$AAR?$AAO?$AAO?$AAT?$AAS?$AA?2?$AAT?$AAo?$AAp?$AAa?$AAz?$AA?2?$AAW?$AAI?$AAN?$AAC?$AAE?$AA6?$AA0?$AA0?$AA?2?$AAP?$AAL?$AAA@ 10004420     Keypad_mx25_topaz_v1:keypad.obj
 0001:000034e4       ??_C@_1CK@CHLCGBHH@?$AAK?$AAe?$AAy?$AAb?$AAd?$AAP?$AAd?$AAd?$AA_?$AAG?$AAe?$AAt?$AAE?$AAv?$AAe?$AAn?$AAt?$AAE?$AAx?$AA2?$AA?$AA@ 100044e4     Keypad_mx25_topaz_v1:keypad.obj
 0001:00003510       ??_C@_1FC@JNHHONNA@?$AAK?$AAp?$AAp?$AAI?$AAs?$AAr?$AAT?$AAh?$AAr?$AAe?$AAa?$AAd?$AAS?$AAt?$AAa?$AAr?$AAt?$AA?3?$AA?5?$AAC?$AAr?$AAe?$AAa?$AAt?$AAe?$AAT?$AAh?$AAr?$AAe?$AAa?$AAd?$AA?5@ 10004510     Keypad_mx25_topaz_v1:keypad.obj
 0001:00003564       ??_C@_1CE@HHBEDKOC@?$AAK?$AAp?$AAp?$AAI?$AAs?$AAr?$AAT?$AAh?$AAr?$AAe?$AAa?$AAd?$AAS?$AAt?$AAa?$AAr?$AAt?$AA?$AA@ 10004564     Keypad_mx25_topaz_v1:keypad.obj
 0001:00003588       ??_C@_1EG@LGAKFIK@?$AA?$FL?$AAK?$AAP?$AAP?$AA?$FN?$AA?5?$AA?$CF?$AAs?$AA?3?$AA?5?$AAf?$AAa?$AAi?$AAl?$AA?5?$AAt?$AAo?$AA?5?$AAB?$AAS?$AAP?$AAK?$AAp?$AAp?$AAR?$AAe?$AAg?$AAI?$AAn?$AAi?$AAt?$AA?$CB@ 10004588     Keypad_mx25_topaz_v1:keypad.obj
 0001:000035d0       ??_C@_1EE@LJPNCNGB@?$AA?$FL?$AAK?$AAP?$AAP?$AA?$FN?$AA?$CF?$AAs?$AA?3?$AA?5?$AA?5?$AAi?$AAr?$AAq?$AA?$DN?$AA0?$AAx?$AA?$CF?$AAx?$AA?0?$AA?5?$AAs?$AAy?$AAs?$AAI?$AAr?$AAq?$AA?$DN?$AA0?$AAx?$AA?$CF?$AAx?$AA?$AN@ 100045d0     Keypad_mx25_topaz_v1:keypad.obj
 0001:00003618       ??_C@_1EI@MFIFPKAO@?$AA?$CF?$AAs?$AA?3?$AA?5?$AAD?$AAo?$AAn?$AAe?$AA?5?$AAe?$AAn?$AAa?$AAb?$AAl?$AAi?$AAn?$AAg?$AA?5?$AAt?$AAh?$AAe?$AA?5?$AAw?$AAa?$AAk?$AAe?$AA?5?$AAs?$AAo?$AAu?$AAr?$AAc@ 10004618     Keypad_mx25_topaz_v1:keypad.obj
 0001:00003660       ??_C@_1FI@DIHGJGMH@?$AA?$CF?$AAs?$AA?3?$AA?5?$AAA?$AAb?$AAo?$AAu?$AAt?$AA?5?$AAt?$AAo?$AA?5?$AAe?$AAn?$AAa?$AAb?$AAl?$AAe?$AA?5?$AAt?$AAh?$AAe?$AA?5?$AAw?$AAa?$AAk?$AAe?$AA?5?$AAs?$AAo?$AAu@ 10004660     Keypad_mx25_topaz_v1:keypad.obj
 0001:000036b8       ??_C@_1FK@POMEHCGJ@?$AAI?$AAs?$AAr?$AAT?$AAh?$AAr?$AAe?$AAa?$AAd?$AAP?$AAr?$AAo?$AAc?$AA?3?$AA?5?$AAK?$AAe?$AAy?$AAb?$AAd?$AAI?$AAn?$AAt?$AAe?$AAr?$AAr?$AAu?$AAp?$AAt?$AAE?$AAn?$AAa@ 100046b8     Keypad_mx25_topaz_v1:keypad.obj
 0001:00003718       ??_C@_1IA@JKNIKOOG@?$AAE?$AAR?$AAR?$AAO?$AAR?$AA?3?$AA?5?$AAF?$AAa?$AAi?$AAl?$AAe?$AAd?$AA?5?$AAt?$AAo?$AA?5?$AAo?$AAb?$AAt?$AAa?$AAi?$AAn?$AA?5?$AAs?$AAy?$AAs?$AAi?$AAn?$AAt?$AAr?$AA?5@ 10004718     Keypad_mx25_topaz_v1:keypad.obj
 0001:00003798       ??_C@_1EK@EALJNCCM@?$AAI?$AAs?$AAr?$AAT?$AAh?$AAr?$AAe?$AAa?$AAd?$AAP?$AAr?$AAo?$AAc?$AA?3?$AA?5?$AAI?$AAn?$AAt?$AAe?$AAr?$AAr?$AAu?$AAp?$AAt?$AAI?$AAn?$AAi?$AAt?$AAi?$AAa?$AAl?$AAi@ 10004798     Keypad_mx25_topaz_v1:keypad.obj
 0001:000037e4       ??_C@_1BM@COLJAECJ@?$AAK?$AAp?$AAp?$AAI?$AAn?$AAi?$AAt?$AAi?$AAa?$AAl?$AAi?$AAz?$AAe?$AA?$AA@ 100047e4     Keypad_mx25_topaz_v1:keypad.obj
 0001:00003800       ??_C@_1GI@JEALIHMP@?$AAK?$AAe?$AAy?$AAb?$AAd?$AAI?$AAs?$AAt?$AAL?$AAo?$AAo?$AAp?$AA?3?$AA?5?$AAK?$AAe?$AAy?$AAb?$AAo?$AAa?$AAr?$AAd?$AA?5?$AAd?$AAr?$AAi?$AAv?$AAe?$AAr?$AA?5?$AAt?$AAh@ 10004800     KeybdIst:KeybdIst.obj
 0001:00003868       ??_C@_1HI@IIIIBLCG@?$AAC?$AA?3?$AA?2?$AAy?$AAm?$AAz?$AAk?$AAi?$AA?2?$AAp?$AAu?$AAb?$AAl?$AAi?$AAc?$AA?2?$AAC?$AAO?$AAM?$AAM?$AAO?$AAN?$AA?2?$AAo?$AAa?$AAk?$AA?2?$AAd?$AAr?$AAi?$AAv?$AAe@ 10004868     KeybdIst:KeybdIst.obj
 0001:000038e0       ??_C@_1BK@BCONKFEE@?$AAK?$AAe?$AAy?$AAb?$AAd?$AAI?$AAs?$AAt?$AAL?$AAo?$AAo?$AAp?$AA?$AA@ 100048e0     KeybdIst:KeybdIst.obj
 0001:00003920       KPPLayout                  10004920 f   BSPKeypad:bspkeypad.obj
 0001:00003a1c       ?BSPKppRegInit@@YAHXZ      10004a1c f   BSPKeypad:bspkeypad.obj
 0001:00003edc       ?BSPKPPGetScanCodes@@YAIQAIQAH@Z 10004edc f   BSPKeypad:bspkeypad.obj
 0001:00004bd4       ?BSPKppPowerOn@@YAHXZ      10005bd4 f   BSPKeypad:bspkeypad.obj
 0001:00004cd8       ?BSPKppPowerOff@@YAHXZ     10005cd8 f   BSPKeypad:bspkeypad.obj
 0001:00004e10       ?BSPKppSetClockGatingMode@@YAHH@Z 10005e10 f   BSPKeypad:bspkeypad.obj
 0001:00004f04       ?BSPKppIsWakeUpSource@@YAHXZ 10005f04 f   BSPKeypad:bspkeypad.obj
 0001:00005108       IL_00000409                10006108 f   InputLang_0409:IL_0409.obj
 0001:00005218       KeybdDriverVKeyToUnicode   10006218 f   LayoutManager:LayMgr.obj
 0001:00007b18       KeybdDriverInitStates      10008b18 f   LayoutManager:LayMgr.obj
 0001:00007b50       KeybdDriverMapVirtualKey   10008b50 f   LayoutManager:LayMgr.obj
 0001:000085d0       KeybdDriverGetInfo         100095d0 f   LayoutManager:LayMgr.obj
 0001:000087b0       KeybdDriverSetMode         100097b0 f   LayoutManager:LayMgr.obj
 0001:000089e0       KeybdDriverPowerHandler    100099e0 f   LayoutManager:LayMgr.obj
 0001:00008aec       ?KeybdEventThreadProc@@YAKPAX@Z 10009aec f   LayoutManager:LayMgr.obj
 0001:00009950       ?KeybdEventCallback@@YAXIIH@Z 1000a950 f   LayoutManager:LayMgr.obj
 0001:00009b2c       ?GetKeyboardProcAddr@@YAP6AHXZPAUHINSTANCE__@@PBG@Z 1000ab2c f   LayoutManager:LayMgr.obj
 0001:00009c54       KeybdDriverInitializeEx    1000ac54 f   LayoutManager:LayMgr.obj
 0001:0000d964       LayoutMgrGetKeyboardType   1000e964 f   LayoutManager:LayMgr.obj
 0001:0000da88       LayoutMgrGetKeyboardLayout 1000ea88 f   LayoutManager:LayMgr.obj
 0001:0000db94       LayoutMgrGetKeyboardLayoutName 1000eb94 f   LayoutManager:LayMgr.obj
 0001:0000dcfc       LayoutMgrGetKeyboardLayoutList 1000ecfc f   LayoutManager:LayMgr.obj
 0001:0000df54       LayoutMgrLoadKeyboardLayout 1000ef54 f   LayoutManager:LayMgr.obj
 0001:0000e790       LayoutMgrActivateKeyboardLayout 1000f790 f   LayoutManager:LayMgr.obj
 0001:0000e968       DllMain                    1000f968 f   LayoutManager:LayMgr.obj
 0001:0000e9f0       SetEvent                   1000f9f0 f i LayoutManager:LayMgr.obj
 0001:0000ea28       GetCurrentThread           1000fa28 f i LayoutManager:LayMgr.obj
 0001:0000ea40       ?wcsrchr@@YAPAGPAGG@Z      1000fa40 f i LayoutManager:LayMgr.obj
 0001:0000ea78       ?wcsstr@@YAPAGPAGPBG@Z     1000fa78 f i LayoutManager:LayMgr.obj
 0001:0000eab0       ?DoProfilerKey@@YAHG@Z     1000fab0 f   LayoutManager:profiler.obj
 0001:0000ec14       NKDbgPrintfW               1000fc14 f   coredll:COREDLL.dll
 0001:0000ec24       Sleep                      1000fc24 f   coredll:COREDLL.dll
 0001:0000ec34       LeaveCriticalSection       1000fc34 f   coredll:COREDLL.dll
 0001:0000ec44       GetTickCount               1000fc44 f   coredll:COREDLL.dll
 0001:0000ec54       EnterCriticalSection       1000fc54 f   coredll:COREDLL.dll
 0001:0000ec64       InitializeCriticalSection  1000fc64 f   coredll:COREDLL.dll
 0001:0000ec74       SetLastError               1000fc74 f   coredll:COREDLL.dll
 0001:0000ec84       DeviceIoControl            1000fc84 f   coredll:COREDLL.dll
 0001:0000ec94       WaitForSingleObject        1000fc94 f   coredll:COREDLL.dll
 0001:0000eca4       SetThreadPriority          1000fca4 f   coredll:COREDLL.dll
 0001:0000ecb4       EventModify                1000fcb4 f   coredll:COREDLL.dll
 0001:0000ecc4       keybd_event                1000fcc4 f   coredll:COREDLL.dll
 0001:0000ecd4       WaitForMultipleObjects     1000fcd4 f   coredll:COREDLL.dll
 0001:0000ece4       StringCchCopyW             1000fce4 f   coredll:COREDLL.dll
 0001:0000ecf4       GetProcAddressW            1000fcf4 f   coredll:COREDLL.dll
 0001:0000ed04       LocalAlloc                 1000fd04 f   coredll:COREDLL.dll
 0001:0000ed14       DeleteCriticalSection      1000fd14 f   coredll:COREDLL.dll
 0001:0000ed24       CloseHandle                1000fd24 f   coredll:COREDLL.dll
 0001:0000ed34       CreateThread               1000fd34 f   coredll:COREDLL.dll
 0001:0000ed44       CreateEventW               1000fd44 f   coredll:COREDLL.dll
 0001:0000ed54       StopDeviceNotifications    1000fd54 f   coredll:COREDLL.dll
 0001:0000ed64       CreateFileW                1000fd64 f   coredll:COREDLL.dll
 0001:0000ed74       ReadMsgQueue               1000fd74 f   coredll:COREDLL.dll
 0001:0000ed84       RequestDeviceNotifications 1000fd84 f   coredll:COREDLL.dll
 0001:0000ed94       GetLastError               1000fd94 f   coredll:COREDLL.dll
 0001:0000eda4       CreateMsgQueue             1000fda4 f   coredll:COREDLL.dll
 0001:0000edb4       RegCloseKey                1000fdb4 f   coredll:COREDLL.dll
 0001:0000edc4       RegQueryValueExW           1000fdc4 f   coredll:COREDLL.dll
 0001:0000edd4       RegOpenKeyExW              1000fdd4 f   coredll:COREDLL.dll
 0001:0000ede4       FreeLibrary                1000fde4 f   coredll:COREDLL.dll
 0001:0000edf4       LoadLibraryW               1000fdf4 f   coredll:COREDLL.dll
 0001:0000ee04       LocalFree                  1000fe04 f   coredll:COREDLL.dll
 0001:0000ee14       RegEnumValueW              1000fe14 f   coredll:COREDLL.dll
 0001:0000ee24       CeSafeCopyMemory           1000fe24 f   coredll:COREDLL.dll
 0001:0000ee34       RegDeleteKeyW              1000fe34 f   coredll:COREDLL.dll
 0001:0000ee44       RegSetValueExW             1000fe44 f   coredll:COREDLL.dll
 0001:0000ee54       RegCreateKeyExW            1000fe54 f   coredll:COREDLL.dll
 0001:0000ee64       StringCchLengthW           1000fe64 f   coredll:COREDLL.dll
 0001:0000ee74       DisableThreadLibraryCalls  1000fe74 f   coredll:COREDLL.dll
 0001:0000ee84       RegisterDbgZones           1000fe84 f   coredll:COREDLL.dll
 0001:0000ee94       ProfileStop                1000fe94 f   coredll:COREDLL.dll
 0001:0000eea4       ProfileStart               1000fea4 f   coredll:COREDLL.dll
 0001:0000eeb4       MmMapIoSpace               1000feb4 f   ceddk:CEDDK.dll
 0001:0000eec4       DDKIomuxSetPadConfig       1000fec4 f   cspddk:CSPDDK.dll
 0001:0000eed4       DDKIomuxSetPinMux          1000fed4 f   cspddk:CSPDDK.dll
 0001:0000eee4       DDKClockGetGatingMode      1000fee4 f   cspddk:CSPDDK.dll
 0001:0000eef4       DDKClockSetGatingMode      1000fef4 f   cspddk:CSPDDK.dll
 0001:0000ef04       _DllMainCRTStartup         1000ff04 f   corelib0:pegdmain.obj
 0001:0000f0ac       __security_init_cookie     100100ac f   corelib0:seccinit.obj
 0001:0000f174       __GSHandlerCheck           10010174 f   corelib0:gshandler.obj
 0001:0000f1bc       __GSHandlerCheckCommon     100101bc f   corelib0:gshandler.obj
 0001:0000f264       __security_check_cookie    10010264 f   corelib0:armsecgs.obj
 0001:0000f278       __gsfailure                10010278 f   corelib0:armsecgs.obj
 0001:0000f2bc       __GSHandlerCheck_SEH       100102bc f   corelib0:gshandlerseh.obj
 0001:0000f344       exit                       10010344 f   corelib0:cexit.obj
 0001:0000f4c4       _exit                      100104c4 f   corelib0:cexit.obj
 0001:0000f4e8       _cexit                     100104e8 f   corelib0:cexit.obj
 0001:0000f504       _c_exit                    10010504 f   corelib0:cexit.obj
 0001:0000f520       GetCurrentProcess          10010520 f i corelib0:cexit.obj
 0001:0000f538       _initterm                  10010538 f   corelib0:crt0dat.obj
 0001:0000f58c       _cinit                     1001058c f   corelib0:crt0dat.obj
 0001:0000f5c8       _onexit                    100105c8 f   corelib0:onexit.obj
 0001:0000f8cc       atexit                     100108cc f   corelib0:onexit.obj
 0001:0000f920       memcpy                     10010920 f   corelib1:COREDLL.dll
 0001:0000f930       memset                     10010930 f   corelib1:COREDLL.dll
 0001:0000f940       towlower                   10010940 f   corelib1:COREDLL.dll
 0001:0000f950       __C_specific_handler       10010950 f   corelib1:COREDLL.dll
 0001:0000f960       __rt_udiv                  10010960 f   corelib1:COREDLL.dll
 0001:0000f970       _wcslwr                    10010970 f   corelib1:COREDLL.dll
 0001:0000f980       wcslen                     10010980 f   corelib1:COREDLL.dll
 0001:0000f990       wcsrchr                    10010990 f   corelib1:COREDLL.dll
 0001:0000f9a0       wcsstr                     100109a0 f   corelib1:COREDLL.dll
 0001:0000f9b0       wcstoul                    100109b0 f   corelib1:COREDLL.dll
 0001:0000f9c0       wcscpy                     100109c0 f   corelib1:COREDLL.dll
 0001:0000f9d0       _wcsicmp                   100109d0 f   corelib1:COREDLL.dll
 0001:0000f9e0       _snwprintf                 100109e0 f   corelib1:COREDLL.dll
 0001:0000f9f0       wcsncat                    100109f0 f   corelib1:COREDLL.dll
 0001:0000fa00       wcsncpy                    10010a00 f   corelib1:COREDLL.dll
 0001:0000fa10       wcsncmp                    10010a10 f   corelib1:COREDLL.dll
 0001:0000fa20       _XcptFilter                10010a20 f   corelib1:COREDLL.dll
 0001:0000fa30       __security_gen_cookie2     10010a30 f   corelib1:COREDLL.dll
 0001:0000fa40       __report_gsfailure         10010a40 f   corelib1:COREDLL.dll
 0001:0000fa50       free                       10010a50 f   corelib1:COREDLL.dll
 0001:0000fa60       malloc                     10010a60 f   corelib1:COREDLL.dll
 0001:0000fa70       realloc                    10010a70 f   corelib1:COREDLL.dll
 0001:0000fa80       _msize                     10010a80 f   corelib1:COREDLL.dll
 0001:0000fa90       ?CSPKppGetIrq@@YAIXZ       10010a90 f   Keypad_mx25_topaz_v1:soc_keypad.obj
 0001:0000faa8       ?CSPKppGetBaseRegAddr@@YAIXZ 10010aa8 f   Keypad_mx25_topaz_v1:soc_keypad.obj
 0001:0000fac4       InterlockedExchange        10010ac4 f   coredll:COREDLL.dll
 0001:0000fad4       TerminateProcess           10010ad4 f   coredll:COREDLL.dll
 0001:0000fae4       InterlockedCompareExchange 10010ae4 f   coredll:COREDLL.dll
 0001:0000fb10       ?KPP_Entry@@YAHIP6AXIIH@ZPAPAUtagKEYBD_PDD@@@Z 10010b10 f   Keypad_mx25_topaz_v1:kbd.obj
 0001:0000fcb4       ?KeybdPdd_PowerHandler@@YAXH@Z 10010cb4 f   Keypad_mx25_topaz_v1:keypad.obj
 0001:0000fd58       ?KppIsrThreadProc@@YAHPAX@Z 10010d58 f   Keypad_mx25_topaz_v1:keypad.obj
 0001:00010068       ?KppIsrThreadStart@@YAHXZ  10011068 f   Keypad_mx25_topaz_v1:keypad.obj
 0001:0001017c       ?KppInitialize@@YAHXZ      1001117c f   Keypad_mx25_topaz_v1:keypad.obj
 0001:000104b8       ?KeybdIstLoop@@YAHPAUtagKEYBD_IST@@@Z 100114b8 f   KeybdIst:KeybdIst.obj
 0001:000106cc       InterruptInitialize        100116cc f   coredll:COREDLL.dll
 0001:000106dc       KernelIoControl            100116dc f   coredll:COREDLL.dll
 0001:000106ec       InterruptDone              100116ec f   coredll:COREDLL.dll
 0001:000107d8       __IMPORT_DESCRIPTOR_COREDLL 100117d8     coredll:COREDLL.dll
 0001:000107ec       __IMPORT_DESCRIPTOR_CEDDK  100117ec     ceddk:CEDDK.dll
 0001:00010800       __IMPORT_DESCRIPTOR_CSPDDK 10011800     cspddk:CSPDDK.dll
 0001:00010814       __NULL_IMPORT_DESCRIPTOR   10011814     coredll:COREDLL.dll
 0002:00000000       __imp_MmMapIoSpace         10012000     ceddk:CEDDK.dll
 0002:00000004       \177CEDDK_NULL_THUNK_DATA  10012004     ceddk:CEDDK.dll
 0002:00000008       __imp_LeaveCriticalSection 10012008     coredll:COREDLL.dll
 0002:0000000c       __imp_GetTickCount         1001200c     coredll:COREDLL.dll
 0002:00000010       __imp_EnterCriticalSection 10012010     coredll:COREDLL.dll
 0002:00000014       __imp_InitializeCriticalSection 10012014     coredll:COREDLL.dll
 0002:00000018       __imp_SetLastError         10012018     coredll:COREDLL.dll
 0002:0000001c       __imp_DeviceIoControl      1001201c     coredll:COREDLL.dll
 0002:00000020       __imp_WaitForSingleObject  10012020     coredll:COREDLL.dll
 0002:00000024       __imp_SetThreadPriority    10012024     coredll:COREDLL.dll
 0002:00000028       __imp_EventModify          10012028     coredll:COREDLL.dll
 0002:0000002c       __imp_keybd_event          1001202c     coredll:COREDLL.dll
 0002:00000030       __imp_WaitForMultipleObjects 10012030     coredll:COREDLL.dll
 0002:00000034       __imp_StringCchCopyW       10012034     coredll:COREDLL.dll
 0002:00000038       __imp_GetProcAddressW      10012038     coredll:COREDLL.dll
 0002:0000003c       __imp_LocalAlloc           1001203c     coredll:COREDLL.dll
 0002:00000040       __imp_DeleteCriticalSection 10012040     coredll:COREDLL.dll
 0002:00000044       __imp_CloseHandle          10012044     coredll:COREDLL.dll
 0002:00000048       __imp_CreateThread         10012048     coredll:COREDLL.dll
 0002:0000004c       __imp_CreateEventW         1001204c     coredll:COREDLL.dll
 0002:00000050       __imp_StopDeviceNotifications 10012050     coredll:COREDLL.dll
 0002:00000054       __imp_CreateFileW          10012054     coredll:COREDLL.dll
 0002:00000058       __imp_Sleep                10012058     coredll:COREDLL.dll
 0002:0000005c       __imp_RequestDeviceNotifications 1001205c     coredll:COREDLL.dll
 0002:00000060       __imp_GetLastError         10012060     coredll:COREDLL.dll
 0002:00000064       __imp_CreateMsgQueue       10012064     coredll:COREDLL.dll
 0002:00000068       __imp_RegCloseKey          10012068     coredll:COREDLL.dll
 0002:0000006c       __imp_RegQueryValueExW     1001206c     coredll:COREDLL.dll
 0002:00000070       __imp_RegOpenKeyExW        10012070     coredll:COREDLL.dll
 0002:00000074       __imp_FreeLibrary          10012074     coredll:COREDLL.dll
 0002:00000078       __imp_LoadLibraryW         10012078     coredll:COREDLL.dll
 0002:0000007c       __imp_LocalFree            1001207c     coredll:COREDLL.dll
 0002:00000080       __imp_RegEnumValueW        10012080     coredll:COREDLL.dll
 0002:00000084       __imp_CeSafeCopyMemory     10012084     coredll:COREDLL.dll
 0002:00000088       __imp_RegDeleteKeyW        10012088     coredll:COREDLL.dll
 0002:0000008c       __imp_RegSetValueExW       1001208c     coredll:COREDLL.dll
 0002:00000090       __imp_RegCreateKeyExW      10012090     coredll:COREDLL.dll
 0002:00000094       __imp_StringCchLengthW     10012094     coredll:COREDLL.dll
 0002:00000098       __imp_DisableThreadLibraryCalls 10012098     coredll:COREDLL.dll
 0002:0000009c       __imp_RegisterDbgZones     1001209c     coredll:COREDLL.dll
 0002:000000a0       __imp_ProfileStop          100120a0     coredll:COREDLL.dll
 0002:000000a4       __imp_ProfileStart         100120a4     coredll:COREDLL.dll
 0002:000000a8       __imp_ReadMsgQueue         100120a8     coredll:COREDLL.dll
 0002:000000ac       __imp_NKDbgPrintfW         100120ac     coredll:COREDLL.dll
 0002:000000b0       __imp_KernelIoControl      100120b0     coredll:COREDLL.dll
 0002:000000b4       __imp_InterruptInitialize  100120b4     coredll:COREDLL.dll
 0002:000000b8       __imp_InterlockedCompareExchange 100120b8     coredll:COREDLL.dll
 0002:000000bc       __imp_TerminateProcess     100120bc     coredll:COREDLL.dll
 0002:000000c0       __imp_InterlockedExchange  100120c0     coredll:COREDLL.dll
 0002:000000c4       __imp_memcpy               100120c4     corelib1:COREDLL.dll
 0002:000000c8       __imp_memset               100120c8     corelib1:COREDLL.dll
 0002:000000cc       __imp_towlower             100120cc     corelib1:COREDLL.dll
 0002:000000d0       __imp___C_specific_handler 100120d0     corelib1:COREDLL.dll
 0002:000000d4       __imp___rt_udiv            100120d4     corelib1:COREDLL.dll
 0002:000000d8       __imp__wcslwr              100120d8     corelib1:COREDLL.dll
 0002:000000dc       __imp_wcslen               100120dc     corelib1:COREDLL.dll
 0002:000000e0       __imp_wcsrchr              100120e0     corelib1:COREDLL.dll
 0002:000000e4       __imp_wcsstr               100120e4     corelib1:COREDLL.dll
 0002:000000e8       __imp_wcstoul              100120e8     corelib1:COREDLL.dll
 0002:000000ec       __imp_wcscpy               100120ec     corelib1:COREDLL.dll
 0002:000000f0       __imp__wcsicmp             100120f0     corelib1:COREDLL.dll
 0002:000000f4       __imp__snwprintf           100120f4     corelib1:COREDLL.dll
 0002:000000f8       __imp_wcsncat              100120f8     corelib1:COREDLL.dll
 0002:000000fc       __imp_wcsncpy              100120fc     corelib1:COREDLL.dll
 0002:00000100       __imp_wcsncmp              10012100     corelib1:COREDLL.dll
 0002:00000104       __imp__XcptFilter          10012104     corelib1:COREDLL.dll
 0002:00000108       __imp___security_gen_cookie2 10012108     corelib1:COREDLL.dll
 0002:0000010c       __imp___report_gsfailure   1001210c     corelib1:COREDLL.dll
 0002:00000110       __imp_free                 10012110     corelib1:COREDLL.dll
 0002:00000114       __imp_malloc               10012114     corelib1:COREDLL.dll
 0002:00000118       __imp_realloc              10012118     corelib1:COREDLL.dll
 0002:0000011c       __imp__msize               1001211c     corelib1:COREDLL.dll
 0002:00000120       __imp_InterruptDone        10012120     coredll:COREDLL.dll
 0002:00000124       \177COREDLL_NULL_THUNK_DATA 10012124     coredll:COREDLL.dll
 0002:00000128       __imp_DDKClockGetGatingMode 10012128     cspddk:CSPDDK.dll
 0002:0000012c       __imp_DDKIomuxSetPinMux    1001212c     cspddk:CSPDDK.dll
 0002:00000130       __imp_DDKIomuxSetPadConfig 10012130     cspddk:CSPDDK.dll
 0002:00000134       __imp_DDKClockSetGatingMode 10012134     cspddk:CSPDDK.dll
 0002:00000138       \177CSPDDK_NULL_THUNK_DATA 10012138     cspddk:CSPDDK.dll
 0002:00000550       dpCurSettings              10012550     LayoutManager:Zones.obj
 0002:0000099c       __security_cookie          1001299c     corelib0:seccinit.obj
 0002:000009a0       __security_cookie_complement 100129a0     corelib0:seccinit.obj
 0002:000009a4       ?g_rgpfnPddEntries@@3PAP6AHIP6AXIIH@ZPAPAUtagKEYBD_PDD@@@ZA 100129a4     PddList_common_topaz_v1:pddlist.obj
 0002:00000b08       ?g_csEventCallback@@3UCRITICAL_SECTION@@A 10012b08     LayoutManager:LayMgr.obj
 0002:00000e68       _exitflag                  10012e68     corelib0:cexit.obj
 0002:00000e6c       ?v_uiPddId@@3IA            10012e6c     Keypad_mx25_topaz_v1:kbd.obj
 0002:00000e70       ?v_pfnKeybdEvent@@3P6AXIIH@ZA 10012e70     Keypad_mx25_topaz_v1:kbd.obj
 0002:00000e74       ?g_dwSysIntr_Keybd@@3KA    10012e74     Keypad_mx25_topaz_v1:keypad.obj
 0002:00000e78       ?g_hevInterrupt@@3PAXA     10012e78     Keypad_mx25_topaz_v1:keypad.obj
 0002:00000e80       __onexitend                10012e80     <common>
 0002:00000e84       __onexitbegin              10012e84     <common>
 0002:00000e88       g_pcsExit                  10012e88     <common>
 0002:00000e8c       _pRawDllMain               10012e8c     <common>

 entry point at        0001:0000ef04

 Static symbols

 0001:00003fec       ?KppScanSequence@@YAIQAIQAHH@Z 10004fec f   BSPKeypad:bspkeypad.obj
 0001:00004f1c       ?KppSaveRegState@@YAXXZ    10005f1c f   BSPKeypad:bspkeypad.obj
 0001:00004fa8       ?KppRestoreRegState@@YAXXZ 10005fa8 f   BSPKeypad:bspkeypad.obj
 0001:00005090       ?KppBusyWait@@YAXK@Z       10006090 f   BSPKeypad:bspkeypad.obj
 0001:00005804       ?LockConfig@@YAXXZ         10006804 f   LayoutManager:LayMgr.obj
 0001:00005884       ?UnlockConfig@@YAXXZ       10006884 f   LayoutManager:LayMgr.obj
 0001:00005908       ?IsLocked@@YAHXZ           10006908 f   LayoutManager:LayMgr.obj
 0001:00005948       ?ValidateInputLanguage@@YAHPBU_INPUT_LANGUAGE@@@Z 10006948 f   LayoutManager:LayMgr.obj
 0001:00005b44       ?VKeyToUnicode@@YAIPAUtagINPUT_LANGUAGE_INFO@@IIPAII@Z 10006b44 f   LayoutManager:LayMgr.obj
 0001:00005e9c       ?GetModifierBits@@YAGPBUMODIFIERS@@PBUMODIFIER_TO_SHIFT@@I@Z 10006e9c f   LayoutManager:LayMgr.obj
 0001:0000602c       ?GetModificationNumber@@YAGPBUMODIFIERS@@G@Z 1000702c f   LayoutManager:LayMgr.obj
 0001:00006114       ?SearchVkToWCharTables@@YAPBU_VK_TO_WCHARS1@@IPAPBU_VK_TO_WCHAR_TABLE@@@Z 10007114 f   LayoutManager:LayMgr.obj
 0001:00006384       ?ProcessModBitsForAttributes@@YAXKIPAGPAPBU_VK_TO_WCHARS1@@@Z 10007384 f   LayoutManager:LayMgr.obj
 0001:00006678       ?GetCharacters@@YAIPAUtagINPUT_LANGUAGE_INFO@@PBU_VK_TO_WCHAR_TABLE@@PBU_VK_TO_WCHARS1@@GIPAII@Z 10007678 f   LayoutManager:LayMgr.obj
 0001:00006b20       ?GetControlledChar@@YAGII@Z 10007b20 f   LayoutManager:LayMgr.obj
 0001:00006b90       ?WriteToCharBuffer@@YAXGIPAI0@Z 10007b90 f   LayoutManager:LayMgr.obj
 0001:00006cc0       ?ProcessDeadKeys@@YAIPAGPBU_DEADKEY@@GPAIII@Z 10007cc0 f   LayoutManager:LayMgr.obj
 0001:00006fa8       ?ProcessLigature@@YAIPAUtagINPUT_LANGUAGE_INFO@@IIGPAII@Z 10007fa8 f   LayoutManager:LayMgr.obj
 0001:00007358       ?KeybdDriverKeyStateToShiftFlags@@YAXQAEIPBU_VK_TO_SHIFT@@1PAI@Z 10008358 f   LayoutManager:LayMgr.obj
 0001:00007548       ?MapLRVKeyToCommonVKey@@YAII@Z 10008548 f   LayoutManager:LayMgr.obj
 0001:000075d8       ?NewKeyStateFlags@@YAIII@Z 100085d8 f   LayoutManager:LayMgr.obj
 0001:00007688       ?AltNumKeyEvent@@YAHIIPAI0@Z 10008688 f   LayoutManager:LayMgr.obj
 0001:00007acc       ?AltNumOkToStart@@YAHI@Z   10008acc f   LayoutManager:LayMgr.obj
 0001:00007e80       ?pKeybdPddInfoFromId@@YAPAUtagKEYBD_PDD_INFO@@I@Z 10008e80 f   LayoutManager:LayMgr.obj
 0001:00007f8c       ?ValidateDeviceLayout@@YAHPBUtagDEVICE_LAYOUT@@@Z 10008f8c f   LayoutManager:LayMgr.obj
 0001:000080c4       ?ScanCodeToVKey@@YAHIPAPAUScanCodeToVKeyData@@IPAI@Z 100090c4 f   LayoutManager:LayMgr.obj
 0001:00008438       ?VKeyToScanCode@@YAIIPBU_VKEY_TO_SCANCODE@@@Z 10009438 f   LayoutManager:LayMgr.obj
 0001:0000855c       ?MapCommonVKeyToLVKey@@YAII@Z 1000955c f   LayoutManager:LayMgr.obj
 0001:00008780       ?VKeyToUnicodeInfo@@YAXPAUKBDI_VKEY_TO_UNICODE_INFO@@@Z 10009780 f   LayoutManager:LayMgr.obj
 0001:0000893c       ?BroadcastToKeyboards@@YAXKPAXK@Z 1000993c f   LayoutManager:LayMgr.obj
 0001:00009230       ?pDLIFromPDDIndex@@YAPAUtagDEVICE_LAYOUT_INFO@@I@Z 1000a230 f   LayoutManager:LayMgr.obj
 0001:000092b4       ?SendRemappedEvent@@YAXIIIHPAUtagDEVICE_LAYOUT_INFO@@@Z 1000a2b4 f   LayoutManager:LayMgr.obj
 0001:00009690       ?Keybd_EventFlags@@YAKIIIH@Z 1000a690 f   LayoutManager:LayMgr.obj
 0001:00009724       ?CallDLRemapFn@@YAIP6AIPBU_KEYBD_EVENT@@IPAU1@I@Z0I1I@Z 1000a724 f   LayoutManager:LayMgr.obj
 0001:00009844       ?WillKeyUp@@YAHIPBUtagDEVICE_LAYOUT_INFO@@@Z 1000a844 f   LayoutManager:LayMgr.obj
 0001:00009a04       ?ToggleLights@@YAXI@Z      1000aa04 f   LayoutManager:LayMgr.obj
 0001:0000a4c8       ?pKeybdPddFromId@@YAPAUtagKEYBD_PDD@@I@Z 1000b4c8 f   LayoutManager:LayMgr.obj
 0001:0000a550       ?ValidateKeybdPdd@@YAHPBUtagKEYBD_PDD@@@Z 1000b550 f   LayoutManager:LayMgr.obj
 0001:0000a580       ?KbdNotificationThread@@YAKPAX@Z 1000b580 f   LayoutManager:LayMgr.obj
 0001:0000ad10       ?SzToHkl@@YAPAUHKL__@@PBG@Z 1000bd10 f   LayoutManager:LayMgr.obj
 0001:0000ae34       ?GetDefaultInputMethodName@@YAHPAG@Z 1000be34 f   LayoutManager:LayMgr.obj
 0001:0000b064       ?GetPreloadInputMethodName@@YAHIPAG@Z 1000c064 f   LayoutManager:LayMgr.obj
 0001:0000b218       ?GetPreloadInputMethodKey@@YAHIPAPAUHKEY__@@@Z 1000c218 f   LayoutManager:LayMgr.obj
 0001:0000b40c       ?OpenKey@@YAHPAUHKEY__@@PBGPAPAU1@@Z 1000c40c f   LayoutManager:LayMgr.obj
 0001:0000b4b8       ?OpenPreloadKey@@YAHPAPAUHKEY__@@@Z 1000c4b8 f   LayoutManager:LayMgr.obj
 0001:0000b544       ?GetPreloadUnNamedValue@@YAHPAG@Z 1000c544 f   LayoutManager:LayMgr.obj
 0001:0000b6e8       ?SetInputLanguage@@YAHPAUHKL__@@PAPAU1@@Z 1000c6e8 f   LayoutManager:LayMgr.obj
 0001:0000bc9c       ?HklToSz@@YAPAGPAUHKL__@@QAG@Z 1000cc9c f   LayoutManager:LayMgr.obj
 0001:0000bdb4       ?IsHklIme@@YAHPAUHKL__@@@Z 1000cdb4 f   LayoutManager:LayMgr.obj
 0001:0000be00       ?GetInputMethodInfo@@YAHPBGPAUtagINPUT_LANGUAGE_INFO@@@Z 1000ce00 f   LayoutManager:LayMgr.obj
 0001:0000c158       ?OpenKeyboardLayoutsKey@@YAHPAPAUHKEY__@@@Z 1000d158 f   LayoutManager:LayMgr.obj
 0001:0000c1e0       ?GenerateModifierToShiftTable@@YAHPAUtagINPUT_LANGUAGE_INFO@@@Z 1000d1e0 f   LayoutManager:LayMgr.obj
 0001:0000c4ec       ?FindVkToShift@@YAPBU_VK_TO_SHIFT@@EPBU1@@Z 1000d4ec f   LayoutManager:LayMgr.obj
 0001:0000c5b0       ?GetImeKeyboardLayout@@YAPAUHKL__@@PAU1@@Z 1000d5b0 f   LayoutManager:LayMgr.obj
 0001:0000c82c       ?SetDeviceLayout@@YAHPAUHKL__@@I@Z 1000d82c f   LayoutManager:LayMgr.obj
 0001:0000cd70       ?GetDeviceLayoutEntry@@YAHPBG0PAPAUHINSTANCE__@@PAP6AHPAUtagDEVICE_LAYOUT@@@Z@Z 1000dd70 f   LayoutManager:LayMgr.obj
 0001:0000cfa0       ?SelectDeviceLayout@@YAHPAGPAUtagKEYBD_PDD@@0K0K@Z 1000dfa0 f   LayoutManager:LayMgr.obj
 0001:0000d43c       ?DeviceLayoutMatchesPDD@@YAHPBG00GPAGK@Z 1000e43c f   LayoutManager:LayMgr.obj
 0001:0000d7fc       ?FormDeviceLayoutEntry@@YAXPBG0PAGK@Z 1000e7fc f   LayoutManager:LayMgr.obj
 0001:0000e5f4       ?IsLayoutLoaded@@YAHPBG@Z  1000f5f4 f   LayoutManager:LayMgr.obj
 0001:0000e6fc       ?GetFirstOpenPreloadIndex@@YAHPAI@Z 1000f6fc f   LayoutManager:LayMgr.obj
 0001:0000ef58       _DllMainCRTStartupHelper   1000ff58 f   corelib0:pegdmain.obj
 0001:0000f368       doexit                     10010368 f   corelib0:cexit.obj
 0001:0000f624       lockexit                   10010624 f   corelib0:onexit.obj
 0001:0000f6c0       unlockexit                 100106c0 f   corelib0:onexit.obj
 0001:0000f6ec       _onexit_nolock             100106ec f   corelib0:onexit.obj
 0001:0000faf4       ?KPP_PowerHandler@@YAXIH@Z 10010af4 f   Keypad_mx25_topaz_v1:kbd.obj
 0001:0000fe44       ?KeybdPdd_GetEventEx2@@YAIIQAIQAH@Z 10010e44 f   Keypad_mx25_topaz_v1:keypad.obj
